:10000000F01F001045380000413800004138000062
:100010004138000041380000413800000000000075
:100020000000000000000000000000004138000057
:10003000413800000000000041380000591600005F
:1000400029140000291400002914000029140000BC
:1000500029140000291400002914000029140000AC
:10006000291400002914000029140000291400009C
:10007000291400003D3800003D3800003D380000E4
:100080001117000029170000411700005917000040
:100090003D380000451800003D3800003D380000A4
:1000A0003D3800003D3800003D3800003D3800007C
:1000B0003D3800003D3800003D3800003D3800006C
:1000C00008B500230B60036000F022FE08BD08B5F0
:1000D0000A20002101F0BCFA08BD08B501F0E8FAD9
:1000E00008BD08B5082002F0A7FE08BD08B5064BFC
:1000F0000020196801F06EFB002001F059FB002080
:1001000001F036FB08BDC046C004001038B50D1C18
:10011000041CFFF7EBFF054B0122291C5A62201C2F
:1001200002F0FEFE002001F033FB38BD640C00102D
:1001300070B5054E051C0E24013C295D301C01F0F4
:10014000A3FD002CF8D170BD743A000038B51648F4
:1001500001F09AFD154C201CFFF7EAFF144D4221D7
:10016000281C01F091FD201C0E30FFF7E1FF432118
:10017000281C01F089FD201C1C30FFF7D9FF0D4819
:1001800001F082FD201C2A30FFF7D2FF281C4E21EF
:1001900001F07AFD201C3830FFF7CAFF616D064878
:1001A00001F072FD38BDC046773A0000C804001067
:1001B0007D3A0000843A00008A3A000010B5041C21
:1001C000FFF794FF201C02F037FE002001F0E0FA58
:1001D00010BD08B50020FFF7F1FF08BD08B5021CEF
:1001E0000249034801F050FD08BDC0469E3A000098
:1001F000963A000013B59620000201F061FB00F072
:1002000013FC154800210322144B00F001FD00F0FF
:1002100015FCFFF7DEFF1248FFF7E0FF002401F0B6
:10022000F3FB002803D001F019F8002409E00A20AC
:1002300001F03EFA684601A9FFF742FF009B002B40
:1002400003D1084B01349C42E9DDFFF7C2FF0648A9
:1002500001F01AFD13BDC046A53A000000000010D1
:10026000B43A00006F170000BA3A000073B5124BA1
:10027000041C1249186803F067FB11490090114AE9
:10028000114B201C01F00BFD00F024FE002812D0C1
:1002900000F03CFEFA218900051C03F055FB061C0A
:1002A000201C01F049FD094B201873430849EB1845
:1002B000321C01F0F4FC73BDC404001040420F0076
:1002C000C53A00009E3A0000D23A000018FCFFFF39
:1002D000D63A000070B5051C0C1C161C00F0A4FBDF
:1002E000291C201C0022064B00F092FC301C01212E
:1002F0000922044B00F08CFC00F0A0FB70BDC0464E
:10030000000000100C00001000B5084B89B01A78EE
:10031000074B68461B78074901F0C1FC694601207C
:10032000054AFFF7D7FF09B000BDC046CC01001059
:1003300008000010E13A0000EF3A000073B5264BC8
:1003400000241D78254B1E78FFF7DEFFFFF741FFE5
:10035000684601A9FFF7B4FE009B002B26D0182B9E
:1003600031D004DC142B0ED0152B1AD106E0352B1E
:100370000BD0842B2DD0342B13D10CE0164B1A78D4
:100380003E2A0ED805E0144B06E0144B1A78062AD4
:1003900007D8013204E0114B1A78002A01D0013A43
:1003A0001A7000F02DFBFFF7AFFF0024009B002B1D
:1003B00002D0C82001F07CF904200121013401F0B1
:1003C00047F91D2CC4DD044B1D70044B1E7000F05A
:1003D00017FBFFF7FEFE73BDCC01001008000010F4
:1003E00010B590B0041C6846FFF740FF69466A46A6
:1003F000201CFFF76FFF10B010BD000073B5182070
:100400000021FFF783FE4C4E4C4D0024983600200F
:1004100001F0BEF94A4B00225A62002C01D00020A4
:1004200000E00620012101F013F9684601A9FFF759
:1004300047FE009B002B23D1002CF0D100F078FD6B
:100440003368002B0DD03F4B00941A6811321A60AC
:1004500004E002F09BFC009B01330093009B102BF7
:10046000F7DD394BED18DCD518200021FFF74EFEE3
:10047000314B94331C6863425C4100F089FACCE74D
:10048000002C06D0182BC2D13048FFF7A7FE00F091
:10049000DDFA009B182B3AD1019B2949002201204B
:1004A00001924862822B24D004DC322B11D0732BB2
:1004B0002AD11BE0872B1FD0C22B02D0832B23D144
:1004C0000CE0234B19680131196002291FD11A6011
:1004D0001DE0204B1B68C01A00F03EFD0120FFF715
:1004E0007FFFFFF776FEFFF7F2FD10E0FFF782FED9
:1004F0000DE0FFF723FF0AE0174B1A70174B052298
:100500001A7000F07DFA02E0019300234B62FFF7BE
:10051000EDFD0098019902F003FD074B94331B6831
:10052000002B03D100F034FA012402E003F024F997
:100530000024024D6BE7C046C804001020BF020033
:10054000640C0010F80200100CFEFFFF033B0000DB
:10055000A401001018000010CC01001008000010C9
:1005600013B501F029FC00F09FFB002004210122BB
:1005700000F09CFE0020021C042100F0E5FE00209B
:100580000521012200F092FE0020021C052100F04E
:10059000DBFE1348002100F0FBFE0021114800F0B3
:1005A000F7FE00F027FC00F065FE2824201CFFF772
:1005B00017FF023CFA2001F07BF8022CF6D101F083
:1005C00037FC02F03FFB1E2300930F2301930648E4
:1005D00006490022064B02F0B1FBFFF70FFFC046B1
:1005E000984004409C400440F9370000C1000000DE
:1005F000F802001000B500E001300378202BFBD09A
:1006000000BD00B5031C303BDAB2092A01D8181C22
:1006100008E020231843031C613B5738052B01D900
:100620000120404200BD70B50E1CFFF7E3FF00251E
:10063000041C06E0FFF7E5FF002805DB2D0105435C
:10064000013420780028F5D13560201C70BD0000F1
:1006500008B500F05BFC011C014801F015FB08BD6A
:100660000D3B000000B5C300181A064BC018072345
:10067000013BC25C002A03D1002BF9D1012000E02C
:10068000002000BD640500107FB5194801F0FCFA98
:1006900000250326354219D1281CFFF7E3FF002867
:1006A00010D0681CFFF7DEFF00280BD0A81CFFF756
:1006B000D9FF002806D0E81CFFF7D4FF002801D09E
:1006C00004350FE00B48291C01F0DEFA291C6846AE
:1006D00001F0D2FB6846FFF72BFD074801F0D4FA82
:1006E0006C1C251CFF2DD5DDFFF730FD7FBDC046FE
:1006F000193B00001E3B0000D77C000070B50E1CAB
:10070000FFF778FF0D25041C2078FFF77AFF0028FB
:1007100007DB01347055013DF6D2201CFFF76AFF5C
:1007200000E0002070BD000030B5464C87B0236863
:100730000868002B06D1444801F0A6FA02F082FABC
:10074000012357E0012B12D10379202B07D0002B76
:1007500005D03E49042201F002FB002803D1394BA9
:100760001A6801326AE03A4801F08EFA5EE00378D6
:10077000412B1BD1374C0230211CFFF7BFFF002853
:1007800054D00378422B51D1211C02300E31FFF797
:10079000B5FF00284AD00378432B47D1211C0230F3
:1007A0001C31FFF7ABFF002849D13FE04D2B23D18F
:1007B000294D0230291CFFF7A1FF002836D003780D
:1007C0004E2B33D1291C02300E31FFF797FF002842
:1007D0002CD00378472B29D1023005A9FFF723FF3E
:1007E000059B002B22DB2A3D6B651C481C4901F050
:1007F0004BFA0023236022E005A9FFF714FF0378DA
:10080000041C202B01D0002B10D10025201C01A995
:10081000FFF774FF0599041C691801A801F040FB5B
:10082000002C03D00135042DF0D108E002F00AFAC3
:100830000A480C4901F028FA024B00221A6007B05E
:1008400030BDC046D4020010273B0000193B000019
:100850003D3B0000C8040010F2040010493B0000BA
:10086000533B0000563B000037B54C6824E0201C89
:10087000FFF7C0FE01A9FFF7D6FE019B041C002B69
:100880001DD0D8B2FF2B09DD00F0DEF9051C019860
:100890000012C0B200F0D8F9019003E000F0D4F9E2
:1008A000002501900198002802D0291CFFF72EFC9A
:1008B00023785A1E9341E4182378002BD7D137BDF3
:1008C00008B5064A012113784B40137001D0044942
:1008D00000E00449044801F0D7F908BDB403001052
:1008E0000A3B00005D3B0000613B000070B5051C49
:1008F00001200821021C00F027FD07240126012009
:100900000821002200F020FD2A1C22413240002054
:10091000022100F019FD01200821021C00F014FD45
:10092000013CECD270BD10B50021041C0A1C022051
:1009300000F00AFD201CFFF7D9FF10BDF7B5012319
:1009400000930023019372B66C46061C02AF01CCE3
:1009500050235B421843C0B2FFF7E5FF0020FFF7CA
:10096000E2FF1020FFF7DFFFE020FFF7DCFF0025AC
:1009700002200021012200F0E7FC705D0135FFF745
:10098000B5FF842DF4D18436BC42E0D162B6F7BD08
:1009900008B5AC20FFF7C7FFAE20FFF7C4FFA520C6
:1009A000FFF7C1FF08BD38B50D1C041C012200F083
:1009B0007DFC291C201C012200F0C6FC38BD08B5B6
:1009C000AF20FFF7B0FFA420FFF7ADFF08BD08B5CB
:1009D000AE20FFF7A8FF08BD10B5041CF820FFF7F4
:1009E000A2FF201CFFF79FFF10BD10B5041C812043
:1009F000FFF799FF3F202040FFF795FF10BD000053
:100A000008B5074B20201B781843FFF78CFF0A20FE
:100A100000F04EFE034B1878FFF7E7FF08BDC04615
:100A200008000010CC01001008B584220248002103
:100A3000520001F061F908BDB503001008B5024885
:100A4000FFF77CFF08BDC046B503001008B50120C4
:100A50000821FFF7A8FF00200221FFF7A4FF0220D2
:100A60000021FFF7A0FF02200621FFF79CFF0320D3
:100A7000011CFFF798FF0320011C002200F064FC1A
:100A800002200621002200F05FFC06210122022044
:100A900000F05AFCFFF7C8FFFFF7D0FFA220FFF7D6
:100AA00042FFA020FFF73FFFC020FFF73CFF0020E0
:100AB000FFF792FF0A2000F0FBFD4020FFF733FF15
:100AC0002C20FFF730FF322000F0F2FD2E20FFF740
:100AD0002AFF322000F0ECFD2F20FFF724FF0A2030
:100AE00000F0E6FDFFF78CFFAF20FFF71CFFA4200E
:100AF000FFF719FF08BD000000B50F290ED88328A5
:100B00000CD8CB08842253430722C0181140044B51
:100B100080220A41111C1A5C1143195400BDC046C1
:100B2000B5030010F0B55B18DBB216E08425CC08E5
:100B30006C4307270F40802504193D41EFB2A618EA
:100B40009C4605E0064BE5182B7801343B432B709F
:100B5000B442F7DB01316346C9B29942E6D3F0BD36
:100B6000B5030010F0B589B0059106921C1C5D68B4
:100B7000DB78834202D22478039444E0A378234AAA
:100B8000C01A0023954209D14300181803234519C0
:100B9000039309E02A7801330232AD188342F9DB6E
:100BA00069782B7803910235EB180026049301969F
:100BB00025E0082F05D1049A954224D02E780027ED
:100BC0000135F30706D5029A069B0798D118C9B2DA
:100BD000FFF792FF0299761001310291013707E089
:100BE000002202920199059A08278B18DBB207931D
:100BF000637802999942DCDB019A01320192019BF0
:100C000003998B42ECDB039809B0F0BD703B000008
:100C1000F0B585B0061C0C1C0292039301F08CF811
:100C200000250190832708E0705D211C029A039B38
:100C3000FFF798FF013024180135A74202D3019B2A
:100C40009D42F1D305B0F0BD00B50F230209184055
:100C50008000031F00D52833002B0EDB511E03201C
:100C6000884280414042002807D1242B06DC042121
:100C70008A1A0349CB18985C00E0002000BDC046EA
:100C8000223F000070B5064E051C0024A05D054BF8
:100C9000291CC018013400F07BFB0A2CF6D170BD72
:100CA0005E3F000000400440F8B51020FFF7EAFF67
:100CB000094C271C143725786678281C311C002223
:100CC00000F0F4FA0234281C311C012200F03CFB35
:100CD000BC42F0D1F8BDC0464A3F0000F8B50B4C0D
:100CE000271C143725786678281C311C012200F057
:100CF000DDFA0234281C311C002200F025FBBC4226
:100D0000F0D10020FFF7BEFFF8BDC0464A3F00000B
:100D1000F0B589B0002404900591FFF7C5FF0220CB
:100D2000072101220694079400F0C0FA022007214F
:100D3000221C00F009FB201C0B2100F0DBFAA04272
:100D400002D11823069301240021264D03916A78CD
:100D50002F78111C0192381C012200F0A7FA381CD0
:100D60000199002200F0F0FA03231F4E029314E0D1
:100D70003078717800F0BEFA002807D103991B4A39
:100D8000A3008A5C183369465A500134029A039BC7
:100D9000013A013302920393023EE30F0021012244
:100DA000A2424B41DBB28B4202D0029B8B42DFDA84
:100DB000381C0199002200F079FA0199381C0122AF
:100DC00000F0C2FA0A4902358D42C0D1201E06D079
:100DD000069B049A05991360079B01200B6009B0DC
:100DE000F0BDC0464A3F0000203F0000223F000007
:100DF0005E3F000008B50120021C0B2100F056FAEE
:100E000001200B21002200F09FFA03200221012281
:100E100000F04CFA03200221002200F095FA08BDF0
:100E200037B5234B10211A68051C8A431A60214BE1
:100E30008022196892010A431A6001200B210022C6
:100E400000F034FA01200B21002200F07DFA1A4B49
:100E50009F211A68194C8A431A601A6818491A6047
:100E6000184B186802F070FD8023000218432A1CFA
:100E700020600221032000F067FA142000F018FC23
:100E80002368FF229343236023680F4A13432360A0
:100E90000E4B1A680192019A002AFADA22680C4B6A
:100EA00013402360FFF7A6FF01980004800D3EBDAC
:100EB00038820440808004409840044000C00140D3
:100EC00000093D00C4040010800000012CC0014056
:100ED000FFFFFFF810B50C4C2068002813DA002043
:100EE0002060FFF79DFF0A280ADC0120FFF798FF2A
:100EF0000138C023FF385B00984201D801232360EA
:100F0000FFF778FF206810BD1400001008B5FFF748
:100F1000E1FF011E08D00120FFF782FF011E03D070
:100F2000024802F011FD011C081C08BD50BB120054
:100F300008B5FFF7CFFF00280AD0FFF7E7FFFA2236
:100F4000031C0021C00FD2009A424841014B186097
:100F500008BDC046D001001010B500280DD0224BAE
:100F600080211A688A431A60204A012311681942B5
:100F7000FCD01F4B03221A6001E01D4B18601D4B73
:100F8000012200211A6019601A6019681142FCD010
:100F9000194B01221A60194A802114684902214321
:100FA00011601A1C002804D10F4B802419682143BA
:100FB0001960134B1968884214D01860002801D0BA
:100FC000104800E01048116802F070FC0F4BFA2145
:100FD0001860890002F0B8FC1E2358430C4B1860BF
:100FE00000F0DAFE10BDC046388204400C80044098
:100FF0007080044074800440788004408080044005
:1010000018000010006CDC02001BB700C4040010C4
:10101000C004001008B500F03BF9134B00211A681A
:10102000120B12031A60114B1A68120B12031A608A
:101030000F4B1A68120B12031A600E4B1A68120B30
:1010400012031A600C4B012219600C4B1A601960D4
:101050001A6019681142FCD0094B23221A60012042
:10106000FFF77AFF08BDC0460080005000800150A5
:1010700000800250008003504080044044800440BF
:101080000880044070B50F490F4800F0FDFD0F487F
:1010900000F0FAFD0E4E0F4D00242B196159DA684D
:1010A000301C0A4B143400F0EFFD782CF5D10A48BF
:1010B00000F0EAFD00F018FB011C084800F0E4FD18
:1010C00070BDC0469E3A0000683F0000BA3F000075
:1010D0007A3F00001C000010853F0000A73F000081
:1010E000F0B53C4B8BB01D68002D3AD03A4B0290C6
:1010F0001B6801209B685DE001342378202BFBD026
:10110000002B3AD0B30008336A469C500136FF2DBD
:1011100001D135E001342378202B01D0002BF9D107
:10112000202B02D1002323700134012E1BD12A4F22
:101130002A4B07223B6001923D1C09E02B68029874
:10114000196800F01BFE002808D02B6814332B60B0
:10115000019B013B0193002BF0D132E03B681D79EC
:1011600001E0041C2E1C2378002B06D0002307224C
:10117000B2425B41DBB2002BBFD1002E1CD000E09D
:101180000025154C022E05D10398154900F0F6FDF7
:10119000002801D0AE420AD823681248D96800F06E
:1011A00073FD23681048196900F06EFD04E02368A0
:1011B000F0B29B6802A99847064B1B68002B07D129
:1011C00003E00198011CFFF75DFF084800F05CFD9B
:1011D0000BB0F0BDD4020010DC0200101C000010A7
:1011E000B43F0000B63F00004E3B0000BD3F000092
:1011F00038B5041C154D0A2808D002D808281CD17F
:1012000010E00D2802D07F2817D10BE02B680022B8
:101210001A700F4800F038FD0E4C201CFFF760FFDD
:101220002C6012E02A680B4B9A420ED90A48211C06
:1012300000F02AFD2B68013B06E00748211C00F066
:1012400023FD2B681C7001332B6038BDD8020010C1
:10125000BA3F0000D4010010C93F000008B503E008
:1012600000F0B0FBFFF7C4FF00F0CEFB0028F7D181
:1012700008BD000008B5034A034B04481A6000F09B
:1012800003FD08BDD4010010D8020010BD3F0000CE
:10129000044B40211A680A431A60034B01221A705A
:1012A0007047C04680800440E002001070B50E4BCD
:1012B000061C1B780D1C141C002B01D1FFF7E8FF46
:1012C000013E022E03D8094BB600F35800E0084B4C
:1012D0001A68012C03D1AC4014431C6003E00124C4
:1012E000AC40A2431A6070BDE00200104C40000008
:1012F0000080005038B50F4B051C1B780C1C002BD0
:1013000001D1FFF7C5FF0020032D11D8281C0123B0
:1013100002F0B8FA02040608074A04E0074A02E0AD
:10132000074A00E0074A1068A3401840431E98414E
:1013300038BDC046E0020010FC3F0050FC3F0150A9
:10134000FC3F0250FC3F035070B50E4B061C1B784F
:101350000D1C141C002B01D1FFF79AFF013E022E39
:1013600003D8094BB600F35800E0084B1A68012C6B
:1013700003D1AC4014431C6003E00124AC40A24301
:101380001A6070BDE002001058400000FC3F0050A1
:1013900038B5084B041C1B780D1C002B01D1FFF73E
:1013A00077FF236818229343236023681D43256039
:1013B00038BDC046E00200101F2342091840012337
:1013C0008340181C014B9200D050704700E100E0B0
:1013D0001F234209184001238340181C2032024B6E
:1013E0009200D0507047C04600E100E0054B3F221C
:1013F0001A60054B01221A60044B40211A688A4387
:101400001A60704724800440D88004403882044029
:1014100008B5044B40211A688A431A60FFF7E6FFBB
:1014200008BDC0463882044008B5154B1868FFF760
:1014300093FD0720FFF7CCFF0820FFF7C9FF0A2024
:10144000FFF7C6FF0C20FFF7C3FF0B20FFF7C0FF1D
:101450000920FFF7BDFF0B4A0023136001210A4A50
:1014600049421160094A1360094A1360094B01227D
:101470001A60094B1A6801321A60C04608BDC0469E
:1014800018000010048204400882044004C0004098
:101490003CC0004000C00040E402001008B5FFF767
:1014A0001DFC0A480021FFF773FF09480021FFF7E0
:1014B0006FFF08480021FFF76BFF07480021FFF787
:1014C00067FF06480021FFF763FF08BD084004409E
:1014D00000400440AC400440144004401C40044020
:1014E000F8B5071C0C1C72B6FFF7D8FF434B1A68FF
:1014F000434B1A60002F01D0424B00E0424B434A5D
:1015000004211360424B434D1A680A431A600023BA
:101510002B609C4218D00720FFF74EFF0820FFF7F2
:101520004BFF0A20FFF748FF0C20FFF745FF0B2079
:10153000FFF742FF384B394A19680A401A602A6897
:10154000EC235B0113432B60002F4FD0344C354903
:1015500000260E60201C311CFFF71AFF301C0921E9
:10156000321CFFF7A3FE301C0921321CFFF7ECFEF2
:101570002D4B8022196811431960236807218B4382
:101580002360236802210B4323607B00DB19990150
:101590005B189B00DF192549254B0F601E60254B0A
:1015A00003211960244B2549186801401960196806
:1015B00009200A431A60FFF7FFFE174A80231168CB
:1015C0009B00194311602A68022113431C4A2B60B7
:1015D000012313601B4A11601B4A124913601660F5
:1015E000136010681842FCD001230B60174B0122D6
:1015F00052421A6062B630BFF8BDC046388204401D
:1016000034820440BF180000FF18000030820440FC
:1016100010ED00E004820440008204407FE2FFFFFE
:101620006440044004C000408080044018C0004072
:1016300008C0004014C000403CC000400FF0FFFF55
:101640007880044070800440748004400882044024
:1016500008B5FFF745FF08BD00B5064B1A68013213
:101660001A601B68013303D1034B1A6801321A60F8
:1016700000BDC046EC020010E802001000B5074BA8
:1016800098420AD8064A00231360064A01381060BF
:10169000054A1360054B07221A6000BDFFFFFF00DB
:1016A000EC02001014E000E018E000E010E000E0C0
:1016B00000B50C4A1368002800D10120C1438B42B9
:1016C00004D809E011688142FCD301E0591C0818D4
:1016D00011689942F6D203E01168C91A8142FBD31E
:1016E00000BDC046EC02001010B5064BFA21186888
:1016F000054B89001C6802F0D9F8044B5C432018A4
:1017000010BDC046EC020010E8020010378941000D
:10171000034B01221A60034B1A6801321A607047AA
:1017200000C00040F0020010034B01221A60034B7E
:101730001A6801321A60704700000140F40200107C
:10174000034B01221A60034B1A6801321A6070477A
:1017500000400140F8020010034B01221A60034BC5
:101760001A6801321A60704700800140FC020010C4
:1017700000B5002803D1044B01221A6003E00128C0
:1017800001D1024B186000BD0440014004800140BB
:1017900000B5002802D1044B186004E0012802D1F2
:1017A000024B00221A6000BD044001400480014049
:1017B00000B5002801D1054B02E0012804D1044BFB
:1017C0001A6802210A431A6000BDC0460440014065
:1017D0000480014010B500280FD1124B80221C68F4
:1017E000920022431A60104B032218600F4B1960BD
:1017F0000F4B1A608022D20211E0012811D1094B4F
:1018000080221868D20002431A600A4B00221A6034
:10181000094B03221960094B1A6080221203084BFE
:101820001A6010BD80800440F8020010184001408A
:1018300014400140FC020010188001401480014057
:1018400000E100E008B5184B1A680E231340062B80
:101850000DD1164B9E221B68DBB2134204D0144AF2
:101860005360144B1B681EE0D9071CD501E0042B04
:1018700005D1104B1868C0B200F0B5F813E00C2B7E
:1018800006D10B4B8022596852000A435A600AE085
:10189000022B08D1054B1A68054B910601D5002291
:1018A00000E001229A6008BD0880004014800040DA
:1018B0000003001000800040004870470003001043
:1018C00070B52B4C2B4B80229203DA67061C00214B
:1018D000201C902200F010FA0023A360264B07255D
:1018E0001A68264CAA431A6019680122114319602C
:1018F000234B1968A9431960196811431960214BDA
:10190000802118684901014319601F4B1A60832226
:10191000226019681D4A1E4B10681B68584301F06D
:10192000C5FF311C000901F0C1FF1A49030A1A4A18
:101930000B60C0B2032310602360184B1D60184B6E
:10194000186860201C680440602CFBD101E014681A
:1019500000E001201C680442F9D1054B01221A70F5
:10196000104B802292031A6005230B6070BDC046A5
:101970000003001004E100E0A44004400C8000409B
:10198000A84004408080044098800440C4040010B3
:1019900078800440048000400080004008800040BF
:1019A0001480004000E100E000B5044A20231168E3
:1019B0001942FCD0024B186000BDC04614800040A4
:1019C0000080004008B5FFF777FF827B031C821878
:1019D000D07B9A7B0132D2B29A7352B2002A01DADA
:1019E00000229A7308BD10B5041CFFF765FF437B06
:1019F000C318DC73437B0133DBB243735BB2002B50
:101A000001DA0023437310BD08B5FFF755FF827B51
:101A1000437BD01A431E984108BD30B5002402E034
:101A20000570013401301D5D002DF9D1121B131C0E
:101A300002E00170013B0130002BFADCD043C017FB
:101A40000240A01830BDF8B5051C0F1C1E1C541E0A
:101A5000092B01D800240FE0181C0A2101F026FFF1
:101A6000221C031C391C281CFFF7EDFF041C2D1839
:101A700005E02F7001340135013A002AF9DC301CF1
:101A80000A2101F057FF30312970601CF8BDF8B50C
:101A90000C1CD9175F18061C4F40551E092F12D970
:101AA000381C0A21002B03DA01F000FF434202E058
:101AB00001F0FCFE031C211C2A1C301CFFF7E7FF71
:101AC000041C351813E0002B00DA951E002201E0FB
:101AD000B4540132A91A0029FADCEC43E4172C4073
:101AE0003519002B03DA2D232B7001340135381CF6
:101AF0000A2101F01FFF30312970601CF8BD73B559
:101B0000069E041C1D1C3009531E00280AD000909C
:101B10001A1C201C2B1CFFF7F2FF241805E0217073
:101B200001300134013A002AF9DC0F231E40092E4E
:101B300001D8303604E0002D01D0373600E05736AA
:101B40002670013076BDF0B585B0041C0F1C00284E
:101B500001D00021017000256BE0252903D0217000
:101B60000132013405E05178252904D12170023277
:101B7000013401355DE0302903D001320292202189
:101B800001E002320292029E9C4632782D3A504287
:101B90004241B6180296002205E00A235A438218F1
:101BA000303AD2B201363078031C303B092BF4D9DD
:101BB0000296AE186346BE4201D97A1BD2B269289A
:101BC0000ED006D863282CD0642809D058283ED1DE
:101BD00019E075280AD078280FD0732837D11AE079
:101BE0001E1D201C1B68FFF752FF04E01E1D201C59
:101BF0001B68FFF728FF331C17E01E1D1B68201C05
:101C00000093002304E01E1D1B68201C0093012389
:101C1000FFF775FFEFE71E1D201C1B68FFF7FDFE99
:101C2000E9E71A68012022700433029A241801326D
:101C30002D181178BD4201D200298ED10023BD425A
:101C400001D2237005E0013C2370013D01E0012534
:101C50006D4205B0281CF0BD10B50C1C131C64218E
:101C6000221CFFF770FF10BD00B5031C9BB00A1CBF
:101C700001A8191CFFF7F0FF632800DDFEE701A8AB
:101C800000F0AAF81BB000BD0FB407B504A901C944
:101C90000191FFF7E9FF03B008BC04B018470EB488
:101CA00003B503AA02CA0192FFF7D6FF02B008BC2F
:101CB00003B0184770B50323041C184205D10D1C4E
:101CC000041C194201D1934201D3002311E0131CDB
:101CD00040CD043B40C4032BFAD8141FA4080134A0
:101CE000A400032309191A400419EEE7CD5CE5545A
:101CF00001339342FAD170BD30B50B040D061D437C
:101D00000D430B021D430323041C93420DD21842C2
:101D10000BD1131C043B20C4032BFBD8141FA408B5
:101D20000134A40003231A400419002301E0E15404
:101D300001339342FBD130BD00B5002300E00133F5
:101D4000C25C002AFBD1181C00BD00B5031C01E0D9
:101D5000013101330A781A70002AF9D100BD30B57B
:101D6000031C002406E01D5D085D281A05D101341E
:101D7000002D02D09442F6D1002030BD00B502E023
:101D80000130002B06D00A78037801319342F7D056
:101D9000981A00E0181C00BD08B5064BFA21186817
:101DA000890001F0D1FDFFF769FC96200002FFF7E2
:101DB00087FD08BDC404001008B5FFF72BF9FFF735
:101DC00067FAFFF725FBFEF741FEFEF72DFEFFF752
:101DD00051FAFFF7E1FF08BD10B5041C02E0013421
:101DE000FFF7E2FD20780028F9D110BD30B5F823C7
:101DF0008A01DB0013404A05920E1343F8221202B7
:101E0000114019430A235943CA1083181C1CEB3490
:101E10005D782478EA336C401B7824021C43835C91
:101E2000201C58400723194008418005800D30BD13
:101E30007047000008B5054B011C984201DD044BBA
:101E4000C1180448EA38FFF7D1FF08BDFF170000AA
:101E500000F8FFFF6440000008B54018511A013136
:101E600001F0D4FD08BD08B5801889189A1A01320E
:101E7000FFF720FF08BD000010B5CB00591A074B33
:101E80000F22C9180023CC5C14400470CC5C0133D1
:101E9000240944700230072BF5D110BD64050010F1
:101EA00010B5CB00591A064BC918002342780478A4
:101EB00012012243CA5401330230072BF6D110BD60
:101EC0006405001030B5B14B87B0D96EB04D4A1ED5
:101ED00091416A46D175A96A1A1CC806400F01389B
:101EE000062807D801F0CEFC040C1F1217191C009D
:101EF000022409E05A6E16329200D3581C1C15E0D9
:101F00005B6E16339B00D45800230FE09B6DD46D9D
:101F1000A3420ADC0AE0022403E00C24032305E0C8
:101F20000D24231C02E00D24EEE70D242C61481142
:101F30001F2800D922E16A461732944901F0ACFC0F
:101F40002000220028002A002D002F003800400029
:101F50004400490051005F0067006F007700850072
:101F60009300A200B400C300D500D300E300E60054
:101F7000E900F100010105010F011101130119012F
:101F8000081C00E08348191C221CFFF765FFF5E0E0
:101F90008148F8E70A1C0E3203E07E4809E00A1C7B
:101FA0001C32081C111C1A1C231C01F0A7F8E5E0C8
:101FB0007948011C0E391A1C231CFFF754FFDDE081
:101FC0007448011C0E31EEE70A1C1C32081C111C5F
:101FD000F1E70A6E1020002A00D00A200A1C0E32F7
:101FE00006E00A6E1020002A00D00A200A1C1C32CB
:101FF00000946C46173402900194081C51E00120B3
:102000001070086E1022002844D00A2242E00A6EA6
:102010001020002A00D00A200A1C0E320EE00120F7
:102020001070086E1022002855D00A2253E00A6E64
:102030001020002A00D00A200A1C1C3200946C4692
:10204000173402900194081C78E00A6E1021002ACF
:1020500000D00A21504A684617300190029100943E
:10206000101C111C1DE00A6E1020002A00D00A204E
:10207000494A00946C46111C173402901C39019493
:10208000101C0EE0096E012010701022002900D0F3
:102090000A22414968461730019002920094081CB8
:1020A000002201F035F869E00A6E1020002A00D005
:1020B0000A20394A00946C46111C173402901C39CE
:1020C0000194101C3AE0096E0120107010220029C2
:1020D00000D00A22304968461730019002920094DD
:1020E000081C00222AE0012010700A6E1021002A2C
:1020F00000D00A21284A68461730019002910094C6
:10210000101C00211AE0009222481CE00092224894
:1021100019E00A6E1020002A00D00A200A1C1C3286
:1021200006E00A6E1020002A00D00A200A1C0E3297
:1021300000946C46173402900194002001F011F8CD
:102140001CE00092081C002104E00D1C1C35081C3A
:102150000092291C1A1C231C01F05EF80EE0081CDA
:1021600002E00C4800E00C48191C221C01F06DF83C
:1021700004E0081C221C191C01F072F86B46DA7D81
:10218000024B07B00120DA6630BDC046C80400101B
:10219000640C0010D6040010E404001010B50649C9
:1021A0000B1C88331A68141C1E34A40060500132C2
:1021B00003210A401A6010BDC8040010054B03201B
:1021C000191C88310A68013A02400A601E329200E6
:1021D000D0587047C8040010F8B5114D2C1C8C3431
:1021E00020680130FFF726FE0E4B0122D8629F6A5D
:1021F000AB6E061C02409A4210D1830703D42068BC
:102200000230FFF7CBFFFF239B001E40B601BF103B
:10221000044B8C35374301222F60DA600220F8BD71
:10222000C8040010640C001030B50C4B0C489A6ABE
:10223000031C8C331C68D3059B0E910500D5403BD5
:10224000856E921001210A40AA4204D1E3188C3015
:102250000360024BD960012030BDC046640C001001
:10226000C804001008B5084B5A1CD07F9A1CD27FB6
:10227000000112021043DA7F0333DB7F10431B039C
:102280001843FFF78BFF08BDC804001038B5FFF7EF
:1022900095FF064903230F22051C5C1815400133E6
:1022A00025770011072BF7D138BDC046C8040010B0
:1022B00008B5FFF783FF034B01228C331860024BF4
:1022C000DA6008BDC8040010640C001010B5064C9C
:1022D000A36E002B06D0FFF771FF044B8C34012254
:1022E0002060DA6010BDC046C8040010640C001005
:1022F00010B5064CA36E002B06D1FFF75FFF044B11
:102300008C3401222060DA6010BDC046C804001081
:10231000640C001008B5104B0022596A1A629142F1
:1023200014D05969914216DD012906D1D96991422B
:1023300003D0DA610A2299615A615A69032A02DDDF
:1023400006490120C866013A5A6104E0044B1B6843
:10235000002B00D0984708BD640C0010C804001082
:102360009003001000B5084B5A6A002A02D05A693F
:10237000002A07DD9A690F21044B1140D977121109
:102380000133DA7700BDC046640C0010C8040010A9
:10239000044B597F9A7F090112020A43197F0A43AD
:1023A0005A677047C804001030B50B1C093B012B5D
:1023B0000FD8084A00239C18257FC45CA54205D08D
:1023C000054B08395A681143596002E001330E2B5E
:1023D000F1D130BDC8040010640C001008B5082904
:1023E0000DD0192913D1427808231A4202D00022B5
:1023F000027002E00F2303700723437005E00023FF
:102400001A1CC25401330E2BFBD1FFF749FD08BD46
:102410001FB50E4B5C6F002802D00F22944304437B
:102420005C67FF2C10DC6846211CFFF725FD684621
:10243000211CFFF7D3FF054A00236C46185D99184D
:10244000013308770E2BF8D11FBDC046C804001019
:1024500030B5124C0F23656F85B09D43054365670A
:10246000082D19D0FF2D17DC6846291CFFF704FD45
:102470006846291CFFF798FF00231A19127F694646
:102480005A5401330E2BF8D16846291CFFF7A6FFDA
:102490006846291CFFF704FD05B030BDC8040010D4
:1024A0001FB50F4C616F082918D0FF2916DC68464C
:1024B000FFF7E2FC616F6846FFF776FF00231A1909
:1024C000127F69465A5401330E2BF8D1616F68466A
:1024D000FFF784FF616F6846FFF7E2FC1FBDC0464F
:1024E000C804001010B50D4C631CD87FA31CDB7F03
:1024F00000011B021843E37F1843E31CDB7F1B032F
:102500001843FFF797FC0F23021C1A402277021191
:10251000134000126377A07710BDC046C8040010B6
:10252000044B5A6E16329200D258121A51424A4146
:10253000DA667047C804001000B5064B5A6E1632B2
:102540009200D1580139D150002901DA0D21D15022
:1025500000BDC046C804001000B5064B5A6E1632C6
:102560009200D1580131D1500E2901D10021D15012
:1025700000BDC046C804001000B5094B5A6E1632A3
:102580009200D2580D2A03D11A1C2932127805E084
:102590009A18507F117F0001021C0A435A6500BD42
:1025A000C804001010B5084B0F245A6E1632920062
:1025B000D1585A6D58181440013104770D2902DCA6
:1025C0005B1812111A7710BDC804001030B50F4BFC
:1025D0005A6E596D16329200D2580D2A07D11C1C22
:1025E00029342478F02008402043586507E09818E3
:1025F000447F057F24012C435C650B114377034B1B
:102600009A180F231940117730BDC046C804001036
:1026100008B504480022011C1C390D23FFF723FCD8
:1026200008BDC0460005001008B504480022011C82
:102630001C310D23FFF717FC08BDC046E404001051
:1026400008B504480022011C1C310D2300F056FD82
:1026500008BDC046E404001008B504480022011C6F
:102660000E390D23FFF7FFFB08BDC046F204001032
:1026700008B504480022011C0E310D23FFF7F3FBBF
:1026800008BDC046E404001008B504480022011C3F
:102690000E310D2300F032FD08BDC046E4040010E9
:1026A0000C4A0023111C46310B70111C47310B7072
:1026B000111C48310B70111C49310B70111C4A312F
:1026C0000B70111C4B310B70111C4C314D320B70C7
:1026D00013707047C804001000B5074A011C04239A
:1026E00000208A1804E0D1184631097840000843D8
:1026F000013BF8D200BDC046C804001030B5074AFF
:1027000000238918012206E0CC18051C4634154028
:10271000257040100133042BF6D130BDC8040010E1
:1027200038B50020FFF7D8FF084C051C0021207F9A
:10273000FFF7E4FF25770420FFF7CEFF0421051CF7
:10274000607FFFF7DBFF657738BDC046C804001027
:1027500010B50020FFF7C0FF034C20770420FFF7DF
:10276000BBFF607710BDC046C804001010B5054C13
:102770000021207FFFF7C2FF607F0421FFF7BEFF2B
:1027800010BDC046C804001010B5094C231C8C3382
:1027900018680130FFF74EFB064B021CD8620F236E
:1027A0001A4022770211134000126377A07710BD00
:1027B000C8040010640C001010B5094C0021201C46
:1027C0000D22FFF749FB201C0E3000210D22FFF7E0
:1027D00043FB201C1C3000210D22FFF73DFB10BDE8
:1027E000C804001010B50C4B00211A1C187F1C786F
:1027F00001312043187701330E29F7D1936E002B56
:1028000008D0064B1B690D2B04D1137F111C2931F5
:102810000B70537310BDC046C8040010640C001048
:1028200010B50C4B00211A1C1C7F18780131204078
:10283000187701330E29F7D1936E002B08D0064B81
:102840001B690D2B04D1137F111C29310B7053739D
:1028500010BDC046C8040010640C00107FB50023F2
:102860000C4A0D251C1C1118097F01306E46995524
:10287000C60F8542664176420133111C30400E2B53
:10288000F1D100236C46185DCA18013310770E2B66
:10289000F8D17FBDC804001010B5074B5A6E163230
:1028A0009200D1585C1801392077D150002901DA03
:1028B0000D21D15010BDC046C8040010034A0023AA
:1028C000111C943198320B6013607047C8040010DB
:1028D000034B012194331A684A401A607047C0467E
:1028E000C8040010044A002313678C321360034BA2
:1028F0000122DA607047C046C8040010640C001062
:1029000008B59C4B0F20996A9B4A8B10184089117F
:10291000013852560E2800D9C5E000F0B3FF081167
:102920001A2327C42EC4C437C4C4C43B3F00002AA2
:1029300000DAB8E0914B9A1840320023937133E0EB
:10294000002A00DAAFE08D4B01209A1840329071D6
:10295000A8E0002A00DAA6E0884B9A184032927963
:10296000DA6621E0081CFFF797FF1DE0002A00DA75
:1029700099E0101CFFF7D4FD16E0002A00DA92E07F
:102980007E4B596E16318900CA500DE0081CFFF7C6
:102990005FFD09E0081CFFF73BFD05E0002A00DAB7
:1029A00081E0101CFFF75AFF01207BE0734B0120F0
:1029B0009833186076E0FFF7DFFDF5E7FFF792FF49
:1029C000F2E7FFF725FEEFE7FFF7ECFDECE76B4BD7
:1029D00000225A66E8E7FFF727FEE5E7FFF7F6FD76
:1029E000E2E7664B012058665CE0FFF729FEDBE773
:1029F000FFF7CAFE022055E0FFF72EFED4E7FFF7EF
:102A000031FCD1E7FFF734FECEE7FFF7D5FECBE789
:102A1000FFF73CFCC8E7FFF737FEC5E7FFF7A2FC6E
:102A2000C2E7564B00221A66BEE7FFF7B1FCBBE7D0
:102A3000524B0120186635E0FFF740FFB4E7FFF77F
:102A40002FFDB1E7FFF744FFAEE7FFF74BFDABE724
:102A5000FFF78CFEA8E7FFF739FCA5E7FFF7C2FEFA
:102A6000A2E7FFF775FE9FE7FFF742FC9CE7FFF741
:102A7000D7FE99E7FFF714FE96E73E4B0120186258
:102A800010E0FFF747FC8FE7FFF756FD8CE7FFF7F5
:102A900047FE89E7FFF760FD86E7FFF709FC83E75C
:102AA0000120404208BD982BBBD03FDC382B98D08A
:102AB0001EDC1C2B00D184E70DDC0C2B00D175E74C
:102AC00003DC0120002BEDD0EAE7162B00D172E7E2
:102AD000182BE5D172E7282B00D178E702DC262BF2
:102AE000DED171E72C2B00D175E7362BD8D175E7F5
:102AF000662B00D186E70CDC4C2B00D178E702DC9A
:102B00003C2BCDD171E7562B00D175E75C2BC7D19B
:102B100075E76C2B00D17BE702DC682BC0D174E732
:102B2000762B00D177E7882BBAD177E7E62B00D157
:102B300097E725DCC82B00D184E70CDCA82B00D15B
:102B400076E702DC9C2BABD16FE7B82B00D173E7A3
:102B5000BC2BA5D173E7D62B00D179E703DCCC2BB6
:102B600000D09DE771E7D82B00D174E7DC2B00D0B3
:102B700096E773E7640C0010647C0000C804001042
:102B8000F32B00D17DE70EDCEC2B00D16FE703DCEB
:102B9000E82B00D084E767E7F12B00D16AE7F22B3E
:102BA00000D07DE769E7F62B00D170E703DCF52B59
:102BB00000D075E768E7F72B00D16BE7F82B00D062
:102BC0006EE76AE738B5184C231C8C331868FFF79A
:102BD00031F9E26E154BA2660022E266DA6003224A
:102BE0009862251C10401C1C022809D090420AD073
:102BF000012802D0FFF784FE07E0FFF7EDFA04E0BA
:102C0000FFF760F901E0FFF70FFB002807DDE3683D
:102C1000002B04D12B1C8C331A6812181A609035C3
:102C20002B681B182B6038BDC8040010640C001002
:102C3000034B0122DA660F229A775A771A77704788
:102C4000C804001010B5054C0549201C00F0DEFE3C
:102C5000FFF7EEFF0123636610BDC046C8040010F5
:102C60009C07000013B50023009301930F4B104CF9
:102C70001A68104B10681968884202D123680093C3
:102C800008E012681A600C4B1B68002B02D06846E3
:102C900001A99847009B2360002B01D0074A93614C
:102CA0005A1E9341064AD36613BDC0469C030010CA
:102CB000AC03001094000010A8030010640C001076
:102CC000C8040010014B4A3318787047C80400103C
:102CD00038B5164B1A1C98321268002A04D0144BCF
:102CE0001D6801231D4001E094331D68114CA36849
:102CF0009D4202D16268002A16D0002D02D1002B1D
:102D00000AD111E00C4B1B68002B02D06168281C13
:102D100098470023636006E0074B1B68002B02D036
:102D2000281C291C9847A56038BDC046C80400105F
:102D300098030010640C0010A003001030B50A4D79
:102D4000049C28600948016009490A60094A136027
:102D5000094B039A1A60094B094A1C60094B1C6015
:102D6000094B1A6030BDC046A0030010A803001034
:102D7000B00300109C030010940300109800001092
:102D8000652C0000640C00109003001008B5084B7F
:102D9000084A196812688A1A1A6006D5FA2252007F
:102DA0001A60054B1A6801321A60FFF791FF08BDDF
:102DB0009C0000109403001098030010F7B50E1C3F
:102DC0000E21051C019200F021FE1A4B03240C2752
:102DD0009E420FDD09236B7301232B7328E0301C07
:102DE0000A2100F007FE301C29550A2100F0ACFD35
:102DF0000134061C002E06D0E30F0022A7425341E7
:102E0000DBB29342EBD1019AA31A033B2B70621BF6
:102E10002B1C01E0195D5973013BD1180229F9D12E
:102E20000F231C1B002301E0013C2B55032CFBDC72
:102E3000F7BDC046FFC99A3BF7B50024124F051CE9
:102E4000261C3B6800960196002B02D0684601A91B
:102E50009847009B0134002B00D000240220FDF78E
:102E60003CF90A4B1A680A4B10681968884208D066
:102E700012681A60FFF78AFF002D02D0013D002D75
:102E800001D0032CDDDDF7BDA80300109C0300106A
:102E9000A4030010F7B51C4D9B235B000E1C1B4ABE
:102EA000E95C1B4BAC5CEB5C002902D00F221440A8
:102EB00002E08021072449009A225200AF5C154AA3
:102EC000CB1AAA5C3435BA1A80277F00791A009190
:102ED00007210C1B013210490194FEF7E0FE00238C
:102EE0000E4F33704124FF35301CFEF725FF2A7842
:102EF0006B783018D31A391C221C0134FEF7CFFE30
:102F0000013D462CF0D1F7BDC80400103701000088
:102F10002F01000035010000747C0000817C00005E
:102F200070B5344B344C1A1C9432126890B0A061C6
:102F3000E161002A17D118280BD1C32909D12F4AE2
:102F400012680F2A05D1181C38300E21162200F005
:102F5000C1F8A369182B04D1E369332B01D100F028
:102F60005FF8FFF765FE0A236361A269244B214DD8
:102F70001A60244B244E1B681A68244B1A600123E4
:102F80002B678C35FFF71EFE2B68B34210D0204A0A
:102F9000934203D01F4A934219D104E0FFF798FEF1
:102FA000FDF79FF813E0FFF793FEFDF790F80EE0B2
:102FB000194C2368002B0AD0684608A9FFF76AFF5E
:102FC0002368684608A998472B6827332B600D4B68
:102FD0001A68124B10681968884203D012681A6088
:102FE000FFF7D4FE034B1B6F002BCBD1FFF770FE16
:102FF00010B070BDC8040010640C001098000010E0
:10300000AC0300109C0300103E2700009400001049
:1030100094330000790D0000B0030010A4030010E9
:10302000F8B5274C002023681D68FFF705FF2368CB
:103030001A689542FCD01E68FFF7FAFD214B0A2260
:10304000214C5A6118229A6101251522DA615D62CC
:10305000231C903300222D361A60FFF7E9FDFF365E
:103060002567174C194D0AE0FFF7ACFD23682A6865
:103070001968914203D01B682B60FFF787FE236815
:103080001B689E42F0D1104D0E4C01262B1C903334
:103090006662182000211F68FFF742FF0C4B381CA6
:1030A000196800F051FC3835011C0422281CFFF778
:1030B00085FE1823A3610023381C6662E361F8BD16
:1030C0009C030010640C0010C8040010A40300103E
:1030D00094030010F0B501240DE005780B1C254089
:1030E00006E0C65CED0077083D43C554351C25401D
:1030F000013BF6D5013A002AEFDCF0BD30B504E023
:10310000845C8D5C85548C5401329A42F8DD30BD6C
:10311000F7B5099D0AAC2678089F2C7894461D1CAB
:10312000002A0DD118E063465B5D4A5DD218131981
:1031300001920024B34201DB9B1B0124435501355E
:10314000BD42F0DD0AE0CA5C12190024B24201DB84
:10315000921B0124C2540133BB42F4DD099B1C7055
:10316000F7BDF7B5099E0AAC2778089D347800288A
:103170002FD000292AD01E1C9446002A0ED1013FD0
:1031800018E063469B5D8A5DD21A131B00240192EE
:10319000A34201DADB19012483550136AE42F0DD8A
:1031A00037E0CA5C121B0024561C01D13A1C0124D2
:1031B000C2540133AB42F4DD2BE0D15C49420C1B1D
:1031C000211E01D0E1190124C1540133AB42F4DDC9
:1031D0001FE000291BD0181C002A06D10EE00E5C4F
:1031E000135C0130F31A1C1BE40FA842F7DD10E05A
:1031F000CA5C0133141B013462425441AB42F7DD17
:1032000007E0D15C013349420C1B611E8C41AB428B
:10321000F7DD099A1470F7BD70B5049D01242C7078
:10322000141C002905D10BE0065D0A5D96420BD106
:1032300001349C42F8DD05E0815C002904D10132B3
:103240009A42F9DD00232B7070BD00B503E04318EE
:103250005B78435401319142F9DB0023435400BDB4
:1032600000B504E08318013B1B788354013A8A427D
:10327000F8DC0023835400BDF0B5114B1A785B785D
:10328000825C1A4000D040220E4C0F49231C261CA1
:1032900004C32C3600221A6001240A1C123117784C
:1032A0005578C75D3D4202D01F6827431F60023238
:1032B00064008A42F3D10433B342EBD10020F0BD65
:1032C00095010010240E0010E100001030B512230B
:1032D0004B43334A0131D3188A0051181A785C786D
:1032E000825C144204D02F4A5F24521894705470A8
:1032F0009A78DC78825C144204D02A4A7C245218E2
:10330000533214701A795C79825C144204D0254AD5
:103310007C245218A33214709A79DC79825C1442AE
:1033200007D0204C5F226418251CA235A1342A70D6
:1033300022701A7A5C7A825C144204D0194A7C2486
:103340005218A03214709A7ADC7A825C144204D04B
:10335000144A7C245218503214701A7B5C7B825CB5
:10336000144207D00F4C5F226418251C523551348B
:103370002A7022709A7BDC7B825C144204D0094A5A
:103380002E245218A43214701A7C5B7C825C134287
:1033900004D0044B5918F43127230B70002030BDA2
:1033A000E1000010940C0010F8B52D4C071C00250E
:1033B000201C20214F22FEF79FFC002D04D0221C50
:1033C0007C23393223701370231C4F3300210135C5
:1033D00019705034052DEBD1214B2D22181C38309B
:1033E0000270181C37300270A1209A705A70400089
:1033F0005F221A541B481A54A320400019541A493A
:1034000008784978385C014204D0191C5331523392
:103410000A701A700024211C381C0134FFF756FF73
:103420000A2CF8D1114D124E00242B786A78FB5CDF
:103430001A4201D0315905E03059FEF77DFC0D49A3
:10344000091A0A310C48043400F0EAFA0235242C37
:10345000EBD10A49084800F0E3FA0520F8BDC04660
:10346000940C00104101000095010010A000001014
:10347000B400001097010010D40D0010897C0000EA
:10348000F0B585B001900027FDF7CEFA6A4C3E1CDE
:103490006A4A7542754113687D19002B00D1D5E049
:1034A000002303AA537023687F210B405C2B00D1BB
:1034B0009EE02BDC382B00D192E013DC072B6CD084
:1034C00006DC022B00D19BE0062B00D0BEE043E0DF
:1034D000212B00D188E0232B00D18FE01C2B00D0C2
:1034E000B4E089E04F2B4ED007DC3F2B64D0402B5B
:1034F00064D0392B00D0A9E066E0542B00D17DE0E8
:103500005B2B3ED0502B00D0A0E06FE0732B69D036
:1035100010DC662B39D005DC5E2B57D0622B00D037
:1035200094E067E06F2B3CD0712B53D06D2B00D013
:103530008CE02CE0792B4BD007DC762B4ED0772B10
:103540003ED0742B00D081E046E07D2B23D07F2B32
:1035500025D07C2B7AD135E031231370022E51DD3A
:10356000231C083B1A687F231A40542A07D0032ED5
:1035700048D0221C0C3A12681340542B42D14C22E2
:1035800006E032233DE033233BE0342339E03522AB
:1035900003AB1A7036E0362333E0372331E03823AB
:1035A0002FE039231370062E2CDD231F1B684722C2
:1035B0001940232926D1EBE7302322E02D2320E0F8
:1035C00041231EE04222E3E74322E1E7442318E0DF
:1035D000452316E0462314E04822D9E7482310E0AB
:1035E0004C230EE050230CE052230AE05222CFE796
:1035F0004F2306E0552304E05522C9E74E2300E09F
:10360000492313700E4B03A8291C0022FDF700FB71
:1036100023681A0605D5E91D0A480022084BFDF764
:10362000F7FA2368DA0572D5E91D07480022044B32
:10363000FDF7EEFA6BE0C046240E0010A401001066
:1036400000000010F53F0000917C0000236801227B
:10365000134206D0A818C0B2002107220223FDF7AA
:1036600061FA23680222134205D0A81DC0B20021CE
:103670000623FDF757FA236804210B4205D0A81D45
:10368000C0B202220623FDF74DFA236808210B423F
:1036900005D0681CC0B207220223FDF743FA236855
:1036A000DA0606D5681CC0B2042102220623FDF703
:1036B00039FA23689A0606D5681CC0B20021022296
:1036C0000623FDF72FFA23685A0606D5681CC0B2F8
:1036D000042107220223FDF725FA23681A0607D5DD
:1036E000281C09300222C0B20821131CFDF71AFA67
:1036F0002368DA050BD5EDB2281C0930C0B20B21C6
:103700000A35FDF7F9F9E8B20A21FDF7F5F90136B6
:1037100004340C370B2E00D0BAE6114B1B68002B7B
:1037200005D01048002109220F4BFDF771FA0F4D0B
:103730000F4E104F0024019A2B78D35C6A781A42FE
:1037400006D0A3009859E15D0922074BFDF760FA06
:1037500001340235092CEED1FDF770F905B0F0BD4A
:10376000D0010010937C00000C000010A00000109D
:10377000A8010010D800001038B5FFF7A3FA002800
:1037800014D006240321201C00F0DEF80321C5B26A
:10379000201C00F02FF9281CC9B2FDF7ADF9092C47
:1037A00001D10B24EEE701340E2CEBDDFDF746F9D9
:1037B00038BD000070B5041CFFF75EFD201CFFF74C
:1037C0005FFE0A4B1B78002B0ED0201CFFF7ECFD90
:1037D000074CC8235B00074EE518211C301C5034F1
:1037E000FEF752FAAC42F8D170BDC046B4030010E7
:1037F000940C00104E3B000000B589B000280ED09C
:10380000FDF7DDF801A80921FEF736FB6846123006
:103810000A21FEF731FB01A8FFF7CCFF08E0FDF716
:10382000D6F8044B1B78002B02D00348FEF72CFA85
:1038300009B000BDB4030010957C000000B5FEE7A0
:1038400000B5FEE708B50A4B0A4A0B4903E01078B9
:103850000132187001338B42F9D3084B084900221A
:1038600001E01A7001338B42FBD3FCF779FEFEE7CF
:1038700000000010EE7C0000CC010010CC01001014
:10388000500E001002B4714649084900095C490015
:103890008E4402BC7047C04603B4714649084000DC
:1038A0004900095A49008E4403BC7047002934D0AE
:1038B0000123002210B488422CD301242407A14202
:1038C00004D2814202D209011B01F8E7E400A142BF
:1038D00004D2814202D249005B00F8E7884201D35A
:1038E000401A1A434C08A04202D3001B5C08224332
:1038F0008C08A04202D3001B9C082243CC08A042A3
:1039000002D3001BDC082243002803D01B0901D08E
:103910000909E3E7101C10BC7047002801D0002003
:10392000C04307B4024802A14018029003BDC0463C
:10393000D90000000029F0D003B5FFF7B9FF0EBC95
:103940004243891A1847C046002941D010B4041CCC
:103950004C40A44601230022002900D549420028FA
:1039600000D5404288422CD301242407A14204D22E
:10397000814202D209011B01F8E7E400A14204D20E
:10398000814202D249005B00F8E7884201D3401A25
:103990001A434C08A04202D3001B5C0822438C0847
:1039A000A04202D3001B9C082243CC08A04202D3B1
:1039B000001BDC082243002803D01B0901D00909A1
:1039C000E3E7101C6446002C00D5404210BC704751
:1039D000002806D003DB0020C043400801E080201F
:1039E000000607B4024802A14018029003BDC04679
:1039F000190000000029EBD003B5FFF7A7FF0EBCAC
:103A00004243891A1847C0467047C04600B500298E
:103A100005D000230139037001300029FAD100BD1F
:103A2000F8B5041CA30719D1231C04CB0F4D104E6D
:103A300050199043021C201C32420FD1181C0B4F0E
:103A400004CBD5199543354208D1181C074F04CB38
:103A5000D51995433542F1D000E001300378002BB1
:103A6000FBD1FEF772F9201CF8BDC046FFFEFEFE3A
:103A7000808080802578000D0A413A200020202592
:103A8000633A20000D0A4D3A20002020473A2025B5
:103A90003032780D0A0025732025730D0A00444D3D
:103AA00031355F530053455249414C20434F4E53EB
:103AB0004F4C45007265616479000D0A4279652EAC
:103AC0002E2E0D0A002573202573202025694D48D0
:103AD0005A0056313500202025692E25303369568D
:103AE000004C43443A25303269202D20256900508E
:103AF0005245535320454E54455220544F20534174
:103B00005645007475726E6564206F6E00424154B4
:103B10003A2025696D560D0A00444D3135000D0AD5
:103B20002530327820200057616974696E672066FD
:103B30006F7220646174612E2E2E0D0A0042616442
:103B4000206D6F64656C0D0A0052656164202573F9
:103B50000D0A004F4B004641494C4544006F6666D4
:103B6000004C43442064656275672025730D0A008C
:103B7000000000005C000C000C7C287C7C447C2451
:103B80001048285408000C00384400443800201025
:103B9000081038108040001010100040002010085D
:103BA000384438007C006454484454281C107C4C31
:103BB000542438542004740C2854280854380050D5
:103BC0000080500010284428282844281004540855
:103BD000384C5C7814787C54283844447C44387CD5
:103BE00054447C14043844347C107C007C00204015
:103BF0003C7C106C7C40407C087C7C047C7C447C5D
:103C00007C14083844787C1468485424047C047C70
:103C1000407C3C403C7C207C6C106C1C601C6454E0
:103C20004C7C4400081020447C00080408808080FC
:103C30000408007844780004040200007F010905AC
:103C40000000070000000000070B064400FF0144CD
:103C5000004400FF01440B0600008C001201FF032A
:103C60002201C40D0782004500250092004801444E
:103C700001820C060000E60019012601C0002001A7
:103C8000070400000000010002080400000000FE1C
:103C90000101020804000000000102FE010B060001
:103CA000008800500020005000880B060000200013
:103CB0002000F80020002006030000000400020B92
:103CC0000600002000200020002000200603000045
:103CD0000000000109050000800160001800060BCB
:103CE000060000FE00010101010101FE08040000C0
:103CF00002000200FF010C060000820141012101C7
:103D000011010E010B0600008200010111011101D9
:103D1000EE0B060000600058004600FF01400B0655
:103D200000009F00090109010901F10B060000FED6
:103D300000110111011101E20B0600000100C10197
:103D400031000D00030B060000EE001101110111FE
:103D500001EE0B0600008E00110111011101FE0899
:103D600004000000008C018C010804000000000029
:103D70000208010A05000020005000880004010B21
:103D8000060000500050005000500050090500008F
:103D9000040188005000200B0600000200010061B1
:103DA0000111000E0D077800860132014902390227
:103DB00042027C0E07800170004C0043004C0070F2
:103DC0000080010B060000FF01110111011101EE3D
:103DD0000B06FE000101010101010101820B06FF3A
:103DE0000101010101010182007C0C060000FF01BC
:103DF00011011101110101010B060000FF01110069
:103E000011001100010C06FE0001010101110191D8
:103E100000F2010C06FF011000100010001000FF5E
:103E2000010804000000000000FF010704C00000BA
:103E3000010001FF0E070000FF01180024004200EE
:103E4000810000010C060000FF01000100010001DB
:103E500000010E07FF010C003000C00030000C0014
:103E6000FF010C06FF01060018002000C000FF0142
:103E70000B06FE000101010101010101FE0B06FF1D
:103E80000111001100110011000E0C06FE000101CD
:103E9000010141018101FE020C06FF011100110028
:103EA00011002900C6010B0600008E00110111014E
:103EB0001101E20B06000001000100FF01010001F9
:103EC0000B06FF000001000100010001FF0D0703C8
:103ED000001C006000800160001C00030D071F0033
:103EE000600080017C00800160001F0E0783014498
:103EF00000280010002800440083010D070300047F
:103F0000000800F00108000400030E0781014101D0
:103F10002101110109010501030100070008000A40
:103F20000100181110133831303378717073C8C123
:103F3000C0C38881808384848782C5C4C7C27574E6
:103F4000777235343732151417120207020802014E
:103F500000030109030402040205030500062024EE
:103F6000282C383C4044484C4669726D7761726534
:103F70002025735F5631350D0A00252D3130732011
:103F800025732573000D0A5479706520273C636FF3
:103F90006D6D616E643E203F2720666F72207061F8
:103FA00072616D730D0A00557074696D6520257519
:103FB000730D0A003F0025730D0A0D0A00564F5974
:103FC00041474552203E3E200025630048656C7005
:103FD000004E6F20706172616D73004B65792070C7
:103FE00072657373003C6B6579313E203C6B65797B
:103FF000323E202E2E2E0044756D70206D656D6F43
:104000007279006C004C6F6164206D656D6F727920
:10401000007400546F67676C6520646973706C612D
:1040200079206F757470757420746F20636F6E7370
:104030006F6C650062005265616420626174746532
:10404000727920766F6C74616765000000800150A2
:104050000080025000800350FC3F0150FC3F0250A2
:10406000FC3F0350EAB820226077373A812A339424
:10407000CFF87C5798A0396BFCF718377F727EBE5B
:10408000AC0F12A47073761C0C817246B11A35D233
:104090007022707C0D6E3C2154F4FAD5EF09B513F3
:1040A000D698FF88360AB8E98A7B197E279230664F
:1040B000871181362D00882542BA65DA4D93BCF907
:1040C00087C900E7720FBCF17B7530EC72B27204E5
:1040D000D1796C11FC24E88D5D48719E680C2F3EEF
:1040E000805D5508C121C9F10CDBCB1700BDB0D7ED
:1040F000049ACF060BE482CFCA6E46445D404D92CF
:104100005EA4D2AD14F3AE437B67EB32A10F57E947
:10411000306DD7637AF2F236A2D11D7B200622CC15
:10412000FE6910607B7445C8FD8DF27985BA4BD26B
:104130008DCD43E4235B0CA07398106E8556849755
:104140001F5D4DBE3ADCAC903A2670BE4DD5AB2417
:104150009881AE730FB84C2E10E18E98EB0E843A16
:104160008C4C49A3B9C53E5417CE9FFD145C310B4E
:10417000F4184C31304204F20433FAB146A61D3E25
:10418000BC798D90F845CECA549F594CDC4A1EDF4D
:1041900041CA20590A457777AB4DA6DC58853806C9
:1041A000B121EDC18B1C0C6347E225038FBEA295A4
:1041B0002938816A21F77B98514899705FED64AB8B
:1041C000C489887CAF5692E9738E01E6688564DF06
:1041D00033FDD82B134ABD8955FBF1CEDABCC9FF9C
:1041E00096FF27960462E3F673F462841EA97BA50A
:1041F0005ECEE20FE483E32F50AC21B7583AF76864
:1042000077BC43C5DA9A215109558BBC3896613188
:104210005CC4BD6D3273DF3AB3085E38712203CBE4
:104220008C8BA7A012E2A454B5A54AEE4EAF3BB9C1
:1042300030FFDAA8C948D73D2A4F14847AFE96C8C1
:104240003E42E61DCF18A02A3C349C480985B3F5B0
:10425000F5C53EC1866D5D432591B139D9522873AC
:104260000DEEC5B673A2B71FA4FCB67A35B8F1F748
:1042700004EB9BF3821250DEDF2AB5240454C07C89
:10428000274628989BFBD40A25B5BCB08F42A624AC
:104290003C913EB885A7C5B66A873BED8F40EDA936
:1042A000FD94405CEBF8D5ECC331B157CFAC7594BD
:1042B0009FD93F8E00D8D925844BD8094E71239AB7
:1042C0003D3545CEC346A74CE959AD26C6463457C1
:1042D000BFBA936A990AA748B1A263FEFC84179DEE
:1042E0008E3F4985008E09FC6BD0CD6DE9A8E5CAEB
:1042F0009C7A1C66077351B0ADAB19F5087BC34BB4
:10430000D81A467F5DAB620AF6C0889836F4A06979
:10431000E31A1925548EC423D6D788C39EA70D0F40
:10432000C71FCF912E37411FB2FB9F8F6697F402B4
:10433000D1EA309A90700885B6BB61020F8692B3BD
:104340003B157367D70BC178D7E9F824E0FD7B668E
:104350005B3E0CFCA76F125EF116EF1AA83DB2DFB0
:10436000242E496EA5A0F16F30F8222818599F6EAF
:104370004873C4AB8F9E7AAF7423B44529E8C6490D
:1043800035FBE2AC559D8293D3898FB6962EC0A89B
:10439000B452CBE2119563C1210EDAF48CBE11A3A5
:1043A0001C14F54FBF23EA8781EEF7E5C21A01CD51
:1043B0009C028519727CD68AF363C962161E515B12
:1043C00047F3525E7498AE048A3CA74C0B8F293891
:1043D000B06F7F28C9F6B1EFC5FA27BBAD3FCB5F01
:1043E00065E4CA7B97A51E3CC0D22D42634F39E9D4
:1043F0008317B6F0E9929CDF988DC71A2DF71483C6
:10440000B153048398131FA173BFD4593FF138727D
:104410001D2651F5AD8FDE747C19E9BEB82AD16C2A
:1044200007663749E54366B092E90B3DE53E8A51A0
:104430000CF0DCFF9DD6E9CFB7FE9E920EFABE5F70
:10444000D653FFD2091EC0A7513A0A2ED45E0F6B75
:10445000CEF711087D7524698DE8C7EFBECB59C929
:1044600083C4D50CE7B8660857FFF9CBB19C0BBEE7
:104470008A504B0B2A37A9F8B0142191F2871A19E8
:1044800010D119DD7AB6D5A3E23B49CEAF298EE82B
:104490001B8209DEF6C2DE3CFBBF9602A3832231FB
:1044A000A36A700FD9AEE6925ED1B48EC95C747FF8
:1044B000BADC7DF5AA74F3A7CF641182B1210E2A6C
:1044C000E25043B825BBAD2CD32FB874168ACB6607
:1044D0005A350724B7B7E64E3FD9789EEF9654BFBA
:1044E000CADBB3BD4585B6146F47B153D8D4175A4C
:1044F000E4F95E777407F24AD8B2073249E1ACFBBF
:10450000423B9C01BBF2809CEB1A8EFEFCF15F9F4C
:104510006D631C1B0B3D953F8AB13E98DC4CFB97AD
:104520009D494D99EE503649E2A396CAA61E5938C8
:1045300096AB20BA671893A4F850C6F7B2866F8777
:10454000A570A895C72732F33D53A82A4D0BED1F40
:1045500036E2EE0025947D7341CE06CEB4CA384BC8
:1045600012FA386E9D40947194F96712F5B91CAF38
:1045700092B6CAF7D3DBDC3947B92DA98EC9D2036D
:104580008720BBEB933877C522F0A76AAB54C66986
:104590001D365E3114D168B59575CCCF2920B28C0B
:1045A0002F4F2C36091A088531251343C930FF0DCA
:1045B0005CBF485543C9210D4BB385454302D17AB1
:1045C000904B2DBAE0EB259752C30A9791DB58C563
:1045D000DA24DFD7B3407C6AAF28E396FAE5663485
:1045E00070A85E3207F6C1191770CA15C5C1B8C5E3
:1045F00060AF0A24A610AD1E554CA0DB57F318DEA1
:10460000E63300230CE5DF5FC30B8D056CB38861D7
:104610007D78C3450D8F937B4D4AAF01218AFE9D66
:10462000DF8456E884F7463C8F90955275CAB8608F
:10463000CE783E5389D974252CAB718058C52DF0A6
:1046400021AF2628AEA88E65D759B317664F1A56E4
:104650003C72B2DA1EF3D07841CEA1C8719A1F0520
:10466000AC7DE6AF01174CBAF98F4781E2BBF78A00
:1046700075E4EF526313325A37A9164FFBA716A2FF
:10468000EA0EDEE4CC39A100A7A659BC77C60A7EA3
:10469000F1B683184243710FB813D4CF8A59272734
:1046A000996EA5BFC5C8273498E6340980D7A76797
:1046B0006E0E41B53B8CD6FD94B5DE4DF99112825C
:1046C000655B03EC6213E9833CD560D2EDBC997E57
:1046D000E38414006EE3C9F143468B2179CBA294A5
:1046E000B9B2B588725E06163FCE83BBBB1A2F994E
:1046F000E46C41089E18B88FBC52F108F8A299BE2C
:10470000A8FF143C32CF2BA099D1BF957C2CF6BFCB
:104710006A210A939441C2A279E9CA4EAF158BCDA2
:10472000E4E5A4CAF070210BFD60CAEDBEE19BCCAC
:10473000D2DF3557822BEA217CA900FE32081B39D3
:1047400023B9D48F6FE7DF5F4F0B893C4387367BFC
:104750008736A009145753E296F84FF12891555126
:1047600036570FBD1143AF3BACB0D850673A26BAAD
:104770006D9AB8337F4CF8F6C9FD9E4CD17564171D
:1047800091343C0A07DEEABE2606D56BF22F4802BA
:104790009C66396501A483C49CBE9E7CC2CD2F1645
:1047A000237FCDFD62637CC8189627121E8A7B5337
:1047B000E586F5D701C258B65995E8DB864A6CF014
:1047C000584197276AD91C46B26C43411987577ADA
:1047D0001A2CD010691B83F4172A445FC2825B94A1
:1047E000C86F3843D500B3E32B1E0CBDBD7C5754B6
:1047F0009E22C055DB5765BB3A1D18AA0BF5A51ABA
:10480000EAA4D5CDC79D53F8B22CE4CF2D25BA67C5
:10481000218EF6D50A1FFAF15844D5034E86BA6F99
:10482000131ABBADA36B09B6E2369DD73ACBDFA412
:10483000B39E78F3C73822B181A224A4ABBE5B3308
:1048400091EFE8A4EDE34F6C1AA773F656DB54A67C
:10485000AB35125268517476E6036CE52B7D6D5FC3
:10486000705619FC9FBBF0540EA3DA97CB85044A0F
:10487000FE8697C7D353CAAE11416DE13EC20A709E
:1048800019A20CECBEFE70D8AB8A37D5CDCFE3C3EE
:10489000CECA27C507B19E8A084B155DF9B17CF0D9
:1048A00059A80C11BEE16EF38D16583F4AF16058BD
:1048B0001D0B79C883B7B59762C3316033D07D577C
:1048C0009F85FA12E587B34F779B07EFBA106B9776
:1048D0000BE1B8EC3029DCDE1055A6E30C19738F20
:1048E000A38E5FD1966D0746B148A2158CAB96ABEF
:1048F00050CAF31C6545568582832B9FE287280C9E
:104900007E61984017F35BF457E930A18B1E222E8D
:10491000E9F506CA59797ABAD4F7FDE668F8E0E411
:104920001935011822A5CB882573B1165FFD8B3A86
:1049300009A85D14400D15CADFCA9B3621D37C63DC
:10494000735417E6BDF3D3D58CCB5B468813F3DBEA
:1049500091D243C6CC6EF91DE6C68DFF7B27F88445
:1049600002ECF44FCFEF5F05069845598AE69D2289
:10497000B3115271074C304364D8EAAA3C7661C047
:10498000548EBD172BCC30B0B0C03A7E45B9C2D3DF
:1049900062D2CD1619B55900515919586C9E11E3C0
:1049A00027DE6E8E3163C6CBB9A27BC502F8F47FD9
:1049B000FBF49443C7C9C82EE13871A353A98E559F
:1049C0003FFE26ADBEFF8A11098BA07FA880F04C68
:1049D0007482FC6B429286CE811796EB348003770B
:1049E0001EB4CBD4E8B27ECB14ED515C3822F0D8A3
:1049F000772C360C70959B86852B9F8CFEC8671D87
:104A000061126D72E6DD282EF01C2F47A85D056F40
:104A100038F524735105810EC73E47C44BA126C00B
:104A200079F44A0683577A9F1A5238F84F771DD186
:104A30009BC8B4CB5A77F6E95D888E8FB82A3F7150
:104A40006AFDE99F8DDF1A8211018DACB0AFC10AFA
:104A500051EDED0A2637CA209E0EBD9830DE128633
:104A600003C160D8BA643C74FDD5CC81EE25F3BC9B
:104A700038278BA16B037551DE2BF94D42F69A6CEA
:104A8000EF2F332B18657B8489252F015E7FECEF98
:104A90008871396073E752C8368F3655F883CEE295
:104AA000B5AC03F655E7FB7836CC75C5C62FA02C00
:104AB0002DD170A5FDE5EAB83763ECADF74519D205
:104AC000BEBBC32BA27D83094F4B1F35E0C89BBFE4
:104AD00074EC48663A62CCCC5B44472F3C98FE1F8E
:104AE00003FF3C1CDC9272489A540D877B6949D6BF
:104AF000845E302938138BD98664EFB1847C07AB90
:104B0000812C733B37DE2A21F3CC0D464E4AF54EFD
:104B10003FA61331673B45A03E49704C2B69536B50
:104B2000A66C2116EE4E5030E1C0A8F7EF3E0F1FE5
:104B3000E626F9198DBCD0980AAA74EF5D28A6095B
:104B400013A87B9F47F55AC38798ED418252ABFC6F
:104B5000B104BCFCB123285D2D8FD02798AD48C38C
:104B6000E11E069B99A8CA4E96002F968CAA762520
:104B7000F197EF652092C601762D383059A267D59E
:104B800087722E8E7C16F662BEABF599A729F2CC01
:104B90005B14376656C7FAC3A47A83699321F2EC93
:104BA00052580D4B7C3BE9AB110ABDBBC4EC9210D3
:104BB000910168FA9C63D610ECCC59264F65E22728
:104BC0006445B03542A515A7E66B07B3F55C1C59E3
:104BD0009CB874E50188278ED8C1AD0C00EA72B28A
:104BE000B6712951C32A96A8A8BADDEFF1A689E0CB
:104BF000C2C28BD190E47C4AB9C2B5CBA3F3BDCB82
:104C0000434FDCF1B00E29D6702B6F4F33B4D70170
:104C1000745F398FC8478024E2D28627DFD964ECDD
:104C20008A28EE6D3C74FF2967059020AF8F54E50C
:104C300054B3789245DD2A532FF3BF3152B8197E11
:104C400093BFA98AED23C23976BA9C2EC514B268E7
:104C5000FF0CD446C47D02BBC6564A875D76185DFC
:104C6000CACDF25FC2FCB5589EA404E33BB57D1DDE
:104C7000E409FFABC389EDEEB2244E6935A71CD918
:104C8000874D4B7AA4CB5F1A70FBB4B9CDFE73038A
:104C9000114E572383B384694A9F9961FFFFEA5AF3
:104CA000470FE5DFD5E74C9DDE4586C13FFDAA7A7B
:104CB000A5123EB0612FFBA665DF87377A459111BB
:104CC00069CBE821A83F2FCA40B975DD4D44EF3AC2
:104CD0003A9842F0EC4D1B4D9996A95689D4E6A11D
:104CE000F28A94EAAB7F7100BA136CC668898B951F
:104CF0002B575B8DD62C63783173B966C103C1BF66
:104D00004222E46FE4990EC39E0E8F6490CF5D76CD
:104D1000B1976B547027E16B9D196762E8504FCED5
:104D2000232FCFF5AF931E54B2FFA9BD49047C21B8
:104D3000B23723B3B296079073263F0847C6F48C68
:104D4000E4F15D182ED26B71ED30E78790F43311EA
:104D500033378EE560B4874F8CBBE13901095116BA
:104D6000C366D6680AA44FA5ADDB05CD7B9B6EC29A
:104D7000530A457C956A778DFF944A42B0A9144640
:104D8000D281F69A51A7FD118D6A86CF2FDB375F4E
:104D90008D11DE7517833D2136424112342912E10F
:104DA0004BC97904C18271F64A93B3C7656CAA3EB8
:104DB0006543B12BF2D37B12FA329BB03F5083C6CE
:104DC00098C3573EA8D2FB0F32A534B21037AF3785
:104DD00049B1BE316D663AAFC70333EB4AEC9EEF83
:104DE0006642037A513DFE10FA848323F7E3ECED2B
:104DF000898234F23E6531D5749535CFBCB073BD30
:104E0000CF43FD1C231AB3A24F4E9A21EE84AD83EB
:104E1000636606FE6EF50B03F88694A1C13915D8BA
:104E20007FB011A4AD0C83CADE3009316C54B712C7
:104E300069364B490A075AFE236138FA8471EF76C6
:104E4000A7038E60273CA9B3F87BC938AA6B9833B7
:104E50005CE9291701DE755AACAA7F4689B7746CE4
:104E6000DB313904FFCE0A1A9845F083469127FFBB
:104E700004F11143CE5FED6BF62FBC3F6845AFB335
:104E8000A01226EA85FC7A1A31618252509BE0F02A
:104E900077E2396F8245765C77BE7BCCBF1EB15915
:104EA000E2E30A005062C22A321490E06F6AC9A39A
:104EB00032214C793E65E8DBAB4197A5109E7AC75D
:104EC000029C7813C66E1D3DF1A172FAFE3A0BBD2D
:104ED000701BC9BF6221C9C9BCAD80F16F4B27E40B
:104EE0001112E40DFAE0F04FAB215E1B1CBC8155A2
:104EF0004C692F58C421AE9041C552A7C41C6AE525
:104F0000A78B5E29F6280CF3206F1150A12F864441
:104F10003B210A3807B16EDE6F0EC3D6CF1454178B
:104F20009732D6FD836B9B73FC360106A5C05FEDFF
:104F3000307144E2067178B706539F150393CCABEA
:104F40007B536C617B6E97B725CADC9D2DDAA8A2D6
:104F5000E44A88AF102376F50108FEB781D5D5B1B4
:104F6000A98BC86BED458895DDA363D6C778036828
:104F70002E45682F3A50919F70E8BA23A761738835
:104F8000BA4F6B677D71328EC0D87BFA337352A7EC
:104F90009A7C8601FE5D16BE07EF4F3AACB93D76AE
:104FA000292588C1B5E18D94EF24621FBA900DF5D3
:104FB000E77D08A52C00782747BBB219D42874C90F
:104FC0000BC0AD0F446F7BE1AB99111FB2F3E06DE5
:104FD000CC03BB8C9E83DD42E5ED4DAEE378C4741B
:104FE000D009D1C756B7843C8BE38042F8F6881FBE
:104FF000A0A3BBF7107E191F4F40756D3CE30D60F9
:10500000D6AF405AB294241E78ABBA3177A505507A
:105010002A63401EE044EF607085FCEA6D3D2AB0D3
:1050200044BBB0126BD47F95F5AAF0460AE57773BE
:10503000931BC50990839DF6F3B445E6B82C1A334B
:10504000836A818AD5EBEE0958FAB7ABDA7D9BC546
:1050500030D2E02C1DA40EF07218EF21C8773C224C
:10506000898D5CED5FE52861D1D4BA181E818F6A05
:10507000B91CDBA87BFFAB6F89622DC5B6F0FC4C79
:105080007E27B396492AF2DD1DB4FBCC6FDBE69197
:1050900025A42A08DD3D8094896D070A0821D7F5EB
:1050A000C280FBFC2393068371074B01B63D022EA1
:1050B000FF2A4131B1DDC33FB805C8088B2706B5CB
:1050C000DFDD75AD7BEFA008C210D8D1D78B54FAC5
:1050D000DA9083B3B36EF946CA7FB16F0B351A6DA0
:1050E000F7435FCD5E6F9156C59C10BF71E02BD426
:1050F0001C2644D524AB4CA58232306FB3CEA64CCF
:105100000F6A42CB504D7D3ABF8A9B28F35C7349AE
:105110004BD2E646F44F239BE7B12A96C3339196D0
:10512000B46F673706E618E8511BAC47551AB983C8
:10513000C5F3ED76FE37BEA59610F3E132386B9CD1
:10514000B6737EA7A2AD094F78C027EDF5B043A78F
:1051500037D7FAA488DEBD2A8D0271165474D53F64
:10516000AF9B5922887B0F6E642E6EDF165548E385
:105170001871AD56F1E496D1F68D9DE42AC9D72E6B
:105180008CC5664600D221201F078FADF2F8F4F5DA
:105190006C0245F10595EFA82135DF479127A19CC9
:1051A0002176163D85A99D2700583217793D8974CF
:1051B000B2FC5248751BA5B3E0F0C9C72BD7B7277F
:1051C000C7A546F0E4AB4B31DE21A61A662D547C10
:1051D00056078A38C7F965383EB25C46725337CDF8
:1051E00076F188D3AD5F404F947403A57B0C56577E
:1051F0006528AF065A8CEFB09E2DAFF57AD66C6954
:10520000E18D77DDE507F84FE294B59B29A704FF10
:105210003811281AA749008BDBADD05765A3293E6A
:10522000F69C94DFF89128B9E9B71621A16AA6ADDA
:1052300091487241B9DDEB3B39A916F15ACC042DE6
:105240003BE167514976556755AFED9F2F7291F657
:10525000944405434A7D3D635EEF3F85DD16F96169
:105260002BC17662CC421651ACAD9DFDC38903982B
:10527000928929BCE6552733D8A3022A44798DD6D2
:10528000417826C3A6CA112DCE2C79461771146A0F
:10529000013232C4410981D32F84F0F4EEEEE8D715
:1052A000A0B4CEB07B4368C8C725A19B1D50DE6962
:1052B00047F0FDA2BF15D3F2B552D1CAB8EBE1EB6E
:1052C000E9821D06A7EC5A82B0723DBE5146CE9EC1
:1052D000FAED95BBCF117E2A9AF7A7ACB71671E409
:1052E000AEFA4B0F253876D7701AAFA1019BFE237B
:1052F000D60BE8D9B5A6461D1DFBAB1A183B0ECE42
:105300008947FB4C9BCC2D675B0372A4A0F43859F2
:10531000F74A9101F487995A6AABD36FF483459D9C
:1053200003B135319A721A5445CD1081D290F5F7F8
:10533000DF605B8D939D4933C97E76EB8C543E8B49
:105340003F47A2ADFC14E3411DE42BC17F3666BD8F
:105350001FEAA84D8CED922A41380BC5996E81AE9B
:105360006F42BB79F4C2C1CB0F8F76DBE66FED9154
:105370002AA97AAB32EA57C59AE6720CD4C171FEFB
:10538000651DCDB7971AEBC44E275935A4AAC08323
:10539000E14D9DC902110E6C4C4B71F0ACA91F92EE
:1053A000250BF4B39B278ADF350017A1A9C6ADC62C
:1053B0005CAA1FCD14187157436D9CDF8E3134B039
:1053C000C4ADB68D1F8DD906BD39A5965CDD238988
:1053D00014525B839C63D67347825CC31C18C78AD4
:1053E000E8A56789AF24AF85CB3A8F47D7A8587116
:1053F00093776B02CCB6A1641A5974F79340F0C945
:1054000029AA5C15C8C5E489CDB6E9C6033D6F324B
:10541000A2030F68F637379416D843D050C1DD6D1C
:105420004F14FBF22646E3989E07B66B8E83F4C4B6
:10543000194461A744FF5BE5F53F08EAAE4CBE2C7A
:105440006B3B9D2851C5C97EE8C12AEEEFA61874B2
:10545000BC726DCD2F03270DCB46C9B699A987A97C
:105460006CC010E617ED71FA61521DBDCAC1E1E0D2
:105470005B7BEF19E10465A09EAF9E5E99D5FB565C
:105480009A7F4426C60D24536CA22CBC1A3194A3D7
:10549000039FCD5AFFAB082478E9161627488FAD35
:1054A0008C258A45F243CFD5E4BA88F9D35D630CE5
:1054B000E16B0BA0E1369ACC6FA82FD3CEA8EA9966
:1054C0003DEEFAACC4A6760AC9B3A2B4233A55633A
:1054D0003F5500496AC99C0E0D949744209A27B203
:1054E000C5858350F098ADE0F04DEE7CBED323C36C
:1054F000BF01F5B4B6767BDCE771EC536ECA5F355D
:105500006BE991CDB330F44FDC55B77EFF8450F892
:10551000DC5B99FD0E858891F8A5EE5355973D17F4
:1055200098ECA106366736AFEDAD81326B4690F050
:105530009D32DC7093EEFA679AA3AB699DAF0CD4F1
:10554000DFB009D2B248EB6AA207309476E824A310
:1055500011BFB9C6911EAFCF86992B966C0297DE0C
:10556000CE183F0152B209FE3ACFD25670153DE631
:10557000B3CA9B1BCF44E69FA46E6EB98EC29689B8
:105580003C6A7CF800C387E84A2553B953BDF6C787
:105590003134923BF3DAE35356D071630B73E91065
:1055A00088CAFCCB8FE84DB676D97D0F7FCBC4DAA5
:1055B000991C3137487CA72110A7C94E67D524B95B
:1055C00034F5D9E3A4C6307A80B2CCAF25C8FB8DC0
:1055D000F986E64B2AB16FB7761BAB11ABE58EE9C6
:1055E000382C02F5BF43230A7A9F057310CC34167A
:1055F000CEEEDE55AE877D975E3552D8042AEFBEDB
:10560000EC3385A1D7E5562071EFD8394595148D37
:10561000F757D38F6087E2C29FF0543AEC7D92FB3C
:10562000EEBF9BF2AD451D3FCED79CCC1D1C393340
:10563000A5D2851D5E0837C912C0EE8778E135D244
:105640006F0B423B8FEE888CAC72BADBFE17688A18
:10565000EB2C3D911DC9777144DEC3D4DC35ABE141
:10566000CBE9824898877962A74F6D4C7BC051B3D4
:1056700092A64EC91081BACE6B333FDA63595EA150
:10568000D3EA21D95E211E8D2D1A444956C00BF351
:1056900051C6F7C221AFFBDCB274995E8C94660CE4
:1056A000179E03B4714A63F26501F7CCED193474A7
:1056B000560A5B81AD89DDCC458DD8AC60C925B576
:1056C0007FE7545A2A1FFB5D05EA1FC25B4E3E105E
:1056D0002B325E05560B724D13E5257516C075A16C
:1056E0004FF476CDD63B833891079A5612E62D5D5E
:1056F000F9E67DE76166ED2B6DFFFA5AE72118E6C2
:10570000E8CDE41ABFBF3B79A1F74FD29D69B63807
:10571000456FEA2A0FCD4461599C1D9CC8DD7B660C
:105720009F24E310DEF79B261E3A5F8A8BF798C80A
:1057300006ECBC242A337C0C9D264B4C9E58B3E1CE
:1057400059D756C05BDD181FEBA109FC86314CED23
:10575000A94029C0AE9C6A04D3BE1FCB5D45D0844E
:10576000AADE89F317FDC7192F62D45260DB571EDA
:105770002E6C08001B21A44B36218B5C4180549376
:10578000D95A2B67A22E0A02956F27D5F6BAD138BF
:10579000DE44FF1BBBDDF7EE2736E50CDFC18DE8ED
:1057A000B3523BDF83D3C669D3B9EE8ADCC2238E02
:1057B000E80D83B39210B2E10A24DF0EAECEFD866F
:1057C0007EBDE670761B7E817D59497A59DBD528EE
:1057D000435CB19BB4FEBDEDA8945FD64391BD4C34
:1057E000008C78918AD86F99B6A5E8D4B09EA906A6
:1057F0003C695218D15392728639FC0233B204E8E4
:1058000093B159BDDE9198E5AAB29B1259F70AE807
:10581000A01E3B20310390B6B81B5C1C9CB2697D76
:10582000148C883831E4F19C494D5534587F95E10A
:10583000A62A096F81376E3B32AFAB651D11A6FCFE
:10584000BEAE4B07CFB4EE91EB05CCF82BEF09EFD2
:10585000B309696AF2135D9A561A9A23B087002633
:10586000EAABC026E404B90B694B659F0345C472DB
:10587000C80B8645227E3939EE2591A6D16D634449
:1058800012D0D2D048BC5E597EABB65F775F3B6327
:10589000C738FDC86089F7A4E2D7710C7565595304
:1058A00051B11BE5CF70026EA9006938DDB5E5A3E3
:1058B0004E705BC332F6D41BFEDA732790396F0E3D
:1058C000056E29871F3EA11E9674743FEE8AE4C0C0
:1058D000039143D6603D1BBD8747346C08463A3080
:1058E000B83338303E1665268701DAAFA68D3D9570
:1058F00096354EC31650E9CFCEEBCAA28342D20BE7
:105900009C0ECF942707EC334F8E12D98CCB3AF1F3
:10591000132C4ED13095DF62E398A6A894064F5B16
:10592000CE3ECA61238E0C47D8BDBBBF7CBC773648
:105930007E9ED0BFC8423A04B2668F19D05396718A
:10594000C54A56DBF78BAC645502257D86D8A1D8B5
:1059500011B24ED136D34044EAAAE889E45111305D
:10596000013CFD2BD50E33A3A104663554CBBE6696
:10597000B6DCD1F5890EB167A322C7E533CE406C02
:10598000778FDCEDAF81CB05FB9B2DE8BB25CD7D73
:1059900012FE7D0BCC389F42CE234D6B3B920AD931
:1059A000E4220B4F6858E9385D6C39AE1B46149EF3
:1059B000181C986E841520FF540DA171ED1F00BEB8
:1059C000B42F9C38BC848BCFE972B1366F8A56FDF8
:1059D000E065E975D8EB6AE3DFE2A91640361DD130
:1059E000FADFFE28CBB5FC4113BE1112F754EC01CF
:1059F000E4C366947C21FD0B4223458C2AC30240FC
:105A0000EEA4EFFE5D819A3864F7FE851E7305B43F
:105A1000EDD3FB61C992DE5F2F777CBFE44936E3AB
:105A2000BF8D5C45DEA0DDB555759680E6DBF606DC
:105A300003B4EC22B3AF7F3EE03402A2ACB75B32DA
:105A400028291AAD27D3D4AA9223672F5EC85702FC
:105A5000AF13A00E3A1E5A9879C882BD63AC6F840A
:105A6000196CF5F6C800AB51CE2C7E8EE8DEDB4219
:105A70007E7C2FA8A9ABD887883812F0B3EEC52951
:105A8000E94F25108E627B928BAD051EFAFA69777D
:105A900049D978F66AE877D605F6970C39D997E5AB
:105AA00010FE47F5F1DCAE1F0E7BBA5C14CB87BC51
:105AB00084710AE609049062B8BDE970DDD4DA4A5F
:105AC000B20F4B3E298F4F60865B46D8002ACA141E
:105AD000EF012BFA243509B6D900CB8DBF5CF594C4
:105AE000C5FA37EC5D80A28B088780A096037D7194
:105AF000663DE8E4FB42D93A1B18C152664EAF68D6
:105B000006CBFC0E97507658D8A2BB94587B368BA8
:105B10007B62CECE77EF87CC56C17F12C3C6E29FA1
:105B2000FB5F054580A2F3E01E869D9167ACC6D55C
:105B3000CA93B7393834B2085246C962C19629C6E9
:105B4000E3FCCF67C2BD52AB7F01E28673B126BBD7
:105B5000A895C76BC6CCFDD1356FBA49AB4E6780EF
:105B60003A92260044D1A3584448CF406B138F6625
:105B70003FD28B6CF81A926B2BAF4FA56C38694FE4
:105B8000096F7462EC10B8FBB98220AB20C16D04C0
:105B9000172D86F28164158CCB84D8103813170C1E
:105BA0004B7ADE9B630B598CD47053017FD54A69C5
:105BB000C74B08E3271CF88CCAA49136A45EF813DF
:105BC0008D47B2EB6C6FB1E5F8B212CCC50E430451
:105BD000A5FEB000FBF0C6357C654E0D18F1B59AF8
:105BE000B93D8891CF936F5D84B5823EC1BB433F81
:105BF000B6DB9B791479E66058DB765C9AA88D64F5
:105C0000D2BDBC7A1B489BDA9397454F80A580E6AE
:105C1000BB2C72B7E0F2D7C094ECEEDCEFD2260BCF
:105C2000CC6193C19A9C4C962A0EE5474D63DE6584
:105C300092A07E77CC3E20F189FBA8740D9B8867EB
:105C400053FECDB282280D0DA9DF389FB1EE3B6A1D
:105C5000BB49AEF32E4E7B8394A706D2CD54E927E1
:105C60009D66E86DDBAB4480E94A86EA1B82784397
:105C700027CF50163B55A1C2A70018EE955692BCEF
:105C80002EED7D97A270FF023C4766FB4388AC90E7
:105C9000210D5D38234C4296A483CE8EB2B99CDC94
:105CA000CD5B20D721CB56CEBA3B8747FCA8ADEAC7
:105CB000A2A5EC0E917349E6A280F642C08560DB96
:105CC000B844FF7E20366869A004F75D4E14544B3B
:105CD0008C2D868261DE767F75728F3F2B527243E8
:105CE00006A4AA18DFB5D4EBAA24D6BCABA58CA910
:105CF00017C93DB3A3F7D9351ACFAB2C45F7E2E767
:105D00009361950D19D7A0362F2CA2B7D103FD436F
:105D10008BAEEA293A5B0E02541EFC1A737C56D0F5
:105D200040F69AAF851E19C13A27B3C7CFD4622374
:105D30000A277E7E00CBD7E1A383B34C9A15D46E9D
:105D4000DDAA08949756944456078966B4F6D3267C
:105D5000DD086D3DC5EDE280794DA8D4A0741843EF
:105D6000DF334C9E4BFE14B5822632109B8B081EEF
:105D70003F0932D32693C180877B9A8FC00385C1A8
:105D80008223FCCBBEE67637328CCE461498992B14
:105D9000DC8D6AD20C432B388FE5B1A5A63A8F2152
:105DA000888793A1EC538025A57635D8468925555B
:105DB0000F194E1A99A3889973E1DCAD6086920B96
:105DC000CF1E6556C1D795D3590DFE4E20539C0D5D
:105DD000BB44B178975D25BE6CD614EC710D4B14A5
:105DE0006D2E9C214BAA954BD3689361B7EFD99444
:105DF000B076AB6A1F642F39F9AE9CBE507EC25399
:105E0000700BB00A9301137DE1F11087328C6D1293
:105E1000D9253CF0C32D5193D200B297FCE3A17178
:105E200063A3D3B083881E03B23FD4CBC48A2E446D
:105E3000474A903D47B3BD584F09C9085BDB24A9C9
:105E400079CE590FBC3C8B94FE093ECF745B402D3C
:105E5000C75567A0610C7B0F6ED131483EC0075D0E
:105E6000A46089834622B541667F80C12D919353FA
:105E7000F23F1208CE441D849F26ED8E767440D3E7
:105E80002C28BA6234A9D060EFC485B4912DFC35BA
:105E9000E4591D29A3CE00687D257CA18CC9A88A60
:105EA000ABA1B0CE76290E060D48219C7AE0D6EF44
:105EB0000C68EC267BABE56292659E83F566175D08
:105EC000A7A70FFBFDB7C11E9190F16CEE9D6BAFC4
:105ED000114CEB68825E9BF35D784C710D5A1D6D21
:105EE000061A79E118A9B045C6D754F6F68690BFD0
:105EF000C9DE04E1DE8F13667D3E8C3378725C8DE3
:105F00009F01C5BCF2B3AA82DD6F43A1E9A0E2FF05
:105F1000ABC760BF48CBC0724BB54542B2D566E84F
:105F2000E59BF65E0E84C44BD46B60FC718A5936D7
:105F3000EDE4EE48069BE9BAC95E10158720176D9F
:105F40002BAB885572B01F04539937C0EB2D050455
:105F5000C3062CBF6BF5C895B132D7DA578E5244C1
:105F60004C89A356595F24BC04B33958C65281AA40
:105F7000D470A3F4140F2E919D93E0A1CC89C1C2DB
:105F80008A816FF7F49A281D73B28F09724C6926C3
:105F90002894CF795F929B9CD5E1087E11672ACB2C
:105FA00077709D4A255517054F1D57A700D88D13AB
:105FB0004D963E15806CE6B2EFC89D48C96EDA4E2C
:105FC000D88F509F8DB51D2ADCC6202BF9F199F78B
:105FD0000ED5F213DEE5B886113CE226FF02CE6153
:105FE0001DFF7F0B108340F66F919B92259BE79BD3
:105FF00023CA5744F983EB9EF2E1DF222B87052A5F
:1060000050BB86F5299094C9321B57DC2E2E88810F
:10601000CC69946B31F0962A9B94FE1C675A84805D
:10602000F91C59CC11D277C29A4281A5E9D21D063A
:10603000F71ED787395C08CA4F57D620C8C3A40DAE
:10604000CDF19F8E40EF92E29A494F889D7D19F3E2
:10605000A0F8BE9ABE5482E9A6CA026482CC149EFD
:1060600047F028A8A1207CA8760BC6DAFFCF351B05
:106070003B704A76852F2F7B373EE66C69AF4882AE
:106080001E5FDEB8B67CD26E0DDB45005F5136B3C5
:10609000897725D518A741DAA25319813309ADE9CB
:1060A0007AB5CDF06D5AF6620E8ED38B06219575BA
:1060B0001E3A947EFAE6F64D91470FFCFED077EF3C
:1060C000622261AC63636FE20E622182EEC913AF9C
:1060D0007836ADA08B419D796D9C0D2A312380B01F
:1060E0002B1AE9CEE0E30902AAD06ABACE7BA960F6
:1060F000964D8CD02D1D220DCF3599C187377660F6
:10610000119C9531FB583102758BD4CB462CF5D8B8
:10611000BD6CB2828B6A5926FD023D222F847649DE
:106120008DAC6407B28E08C8CB69892B34014D321F
:10613000D3820A620C9D2138FA52E6EAB0B855BC07
:10614000D901A087607155C63A0E45F4B4422122A8
:1061500038E0573C44C3D6FECF18165E466C01B5F6
:106160009993F63A617CC1AC29241F2EBE3FAD6CD9
:10617000926ECCE26C7019C72C9AE909E5CEFB034C
:106180008153BDEF78803240A3D75A7787C7B8E6EE
:10619000F6EAB102CB8A42ADE4B50C20EA8EC8B76C
:1061A000AE422DBFE453615C0FACEEBDF2186E0938
:1061B000967F02B2B10B40D91D2621B6994CDB2542
:1061C0001818E888D384A1618ADE376A410109C1C1
:1061D000EB65E0862ACEDB2DAEE5564F8BC0A5A938
:1061E000B9EA3F2E1D15BA14F6C092949AD1C4593B
:1061F00075BA8F15E54EF99C051314D3BF03C9C2B8
:106200007F826541B7BB87BD67BD6B29668685A761
:10621000AC28EB194813D4EE2ED1DEC30D5C0F0071
:1062200053B0E47B97EAB1BC7B3621AACFEFE49070
:10623000B54E959FB534FE5C58A0A7477E747C226E
:10624000D7EED09C0321CFA11A1153985222B30844
:106250000C28CBC39196E2B425EFD12E28337B9E38
:10626000A9F39A9BF9B7DF1AFF0D254B7997A51D66
:10627000AA9B2A94DAF3DBFE841BBB1AB32076EECA
:10628000CBB5D83D34B1F69E88F3AC4642377CC6D8
:106290000620BFAC2F31FA942A24387CBE84B50284
:1062A0004ED59ACFEDB0D7ECD4A20956E84950C7E5
:1062B0000FF168D4CDC4A16B00ED0115980419FE4F
:1062C000966CA4FBF7BE2983DF2999FB0D02951D6F
:1062D0006AF04C4DD110D28D5D7BE78EF55CD54CCC
:1062E000FDBEBB65DBCBD97A79B27E5D83D3759772
:1062F000099A27AFCD39F6BE0184D6964D9F532F0C
:10630000A9576CC5B0E1FBB9A8BE5DF163035FFAA4
:10631000E9885C3CA9BED3E6C4ABB184DE1330008F
:106320003014CB2493595D6442A65AED9C148FF12E
:10633000A91904A0611BCB602B0B31CF4EF08DD679
:1063400023B8BFE4182AC0D1A0B011A30A09940849
:10635000E3BAF882663B8B675B0D5242B89EF583C9
:106360009999A335CA12326895133A15F71EBCD114
:10637000459FABDA4FC6CA1C62B69423BE24B6341E
:10638000FE8484302EFD27052FC0C795B193CCBB6A
:10639000C7C3546C88FF419C5BC323B0F3D6C9D4F8
:1063A000110BC6C5392D7888BAE8F7368DF9CB06BA
:1063B00070EFF033194738049B9DAA420E31A47543
:1063C000C0C4E0433310601F35F7FF7693289ADA94
:1063D000874DB5B27FD71A93A19AB4159B9D053E00
:1063E000EAB6DB2F5A43E99F5224016FACCEBB3F84
:1063F000FE1A54BFEA0C755FC7ED79501F04FFB851
:10640000FE974790DC1E8B5858BD4805FB06137954
:10641000DC6C60FB7BAC1622CB30F8A217E02DDBE6
:10642000CF70388FD5510F133EF40D4011F879A677
:10643000C19DDC3FCBB854F14FB08AC300D3165A8C
:10644000CB87151D7A02B8DFFFD78502FD5CDBEA3A
:10645000EBAAB4EB78C572169E595153A07BC323A7
:106460001BE482F6E4AEA93832B6718018EA6CE417
:106470003D6391321725A2B20BC746809856485407
:10648000182D435739E6B5224257784B82C33D2237
:10649000D0B18EE9F0A72C756C9F920DD5333621C3
:1064A000E30C06A6D7B78A626C00C1658FF3701043
:1064B0002157A6F2C7D7BC695EFAD145CB39C7547C
:1064C000922C5B8CB711D721753D57BDEC57DBCDB6
:1064D000B0BDCA688BCE5C90B978D68BC5ED999467
:1064E000149C854505F4FF93FE4DE163C4CF8DA157
:1064F000FBF3BA51C4B4192D3CF908907AE9A2E033
:106500008D3EE8B0B8561683CDBC477867D13E0AB9
:10651000D71529A45DC6F6A0E0676C8390571AAB27
:106520008AC1337009829132FD8AE7232D9E791248
:10653000240B747CD1BAC798D12FEFD876DE6DFDCD
:10654000B32D1F1A00922229203AF874E3D7609ADB
:106550002C70ABC56786D3EE24D42FF9B8118324F1
:10656000E6C055EB82839FE64C5A35D570F7FFECB9
:10657000899F6055C65A26D7BB81B9092C6CAB7F61
:1065800002758D0F4580E667D9DBF0EC208CB19E5B
:106590000B0D281F68F10CE47EAC459DAED0A6D74C
:1065A0002D5B7F6B21A5DA7B4F6C132414924B017A
:1065B000F30385B952B2C8A7E92EA0BD56529A5727
:1065C000679275664F268B1D49FB8511BE1435D524
:1065D00085331389E75BE8CCC9ACD9E93A4FD810C9
:1065E000D91913DB129198823AD17FDEA9C23046C5
:1065F00097401B347F2C14C7B6B34D34532CDF00A7
:10660000BE97A8646DBDFFC6F2A8B4C126D24EC81D
:1066100012FCDECBEDB7455B78D60933347E95AFFF
:106620009259139AB620B5CC74ED5BD82CE7DAD426
:10663000DECEAE11DFCD61C17016EC6199E75CC2B0
:106640004BF2461DAA75BB33CA6420C81923029CAD
:1066500098F684DCD3D12C7F0FEC829F2E79245EB8
:106660002269378F3258C46DA9F06B8DB48B5F905F
:10667000DAC7D74A146999CEFBBD967DEA27EB129B
:10668000602B7E5482119EF6F0BAC49034B9B0B536
:106690005B33DCE4E3261BD1C339375B845873B129
:1066A00080B9A10E62087FCA83B36292F9B24869C9
:1066B00094F3D25E2A5886B7E9BB8736F056B33FCB
:1066C00085EE939427D54AC1E33B7DA1601915ACB3
:1066D00003BB32D1F26AFC8942E217EE343AF7A8E2
:1066E00042C795F23730AD29B1C04C56BC28296F4E
:1066F000FED67A98B748306C480627FC39B86F91B7
:1067000067957FA28BE63A9F9E6BB719E791B20916
:10671000F5ECF06E4C96A4EFDDF8703EA31A1C5118
:1067200011D9411642F11BEF7E3A3F4D04317355AA
:10673000B9FBCCE898DA1042ECE419729726F153D1
:1067400067264B61D2AF2909141D1F69FBB5E6D03E
:10675000FFD33992AF8B0CB0DB22B32FD69B0D0742
:10676000E9F61AF928ED4AA098127C5B9F736AF744
:10677000DC37FBBACA71E6ADD678E821D1CE67A284
:106780000E8EE7F042DECC0702450BB13D191A9898
:1067900056E907914496DDF9BB0F8EF3F12EE652D0
:1067A0009A5912D9253F0DA0D8FF4ED644D62DC9EF
:1067B000D461E9366D786AC50CBCE9FBD9FEBECA66
:1067C000136748E24F173D3E0F24C640DDEA6E389E
:1067D0002C2193484C479438336F6FF504965381BE
:1067E00073047914A4C156DD06A558952A2B6DAC07
:1067F00080517509907FA791D35F22E2A96C4B2845
:10680000350E8A48CF7EA79F5456B954553846CC8A
:106810002C7B4E3AF1B50F3A2D64897AD4CA108E8A
:10682000C3250FD521B3140FFDABEC2ED49FD07E22
:106830003D2B9851FF6737F166D9C1D39172299EDC
:10684000280E1BE00634BE788203CD8EFBE2B193A6
:10685000EE8899D634A5F5F173D02446D7BA56ED13
:10686000766FDD78E6611006625C84E6AD405926FD
:10687000C9D4ECB658DE1B85EAEA6B64591FA470D4
:10688000DB450B4341F89748D4D199C5D4514034E6
:10689000277C2CBE046EAA44FFD103D9E9D728086F
:1068A0000C27CE89E2EC42F283C589EC230472B155
:1068B00014FEC22E9A038BFEA6B361413943F2BE89
:1068C000E679108F3CFAA3ADF590E2905AF2832E50
:1068D000D8F61FE5D888A55BD71F88B66965706FA5
:1068E000B9B7319D37F28E7807A28B7E6EC9C55736
:1068F00047A410DA78BA69D016CC2EB72EAA4C85E8
:10690000F608A972EB3B97CF88C02B438AC31D4181
:10691000A205D6513AA0D79148E772E1D2BF4CE721
:10692000AEC8CA35CFBC45DCE9473CA0CB68003FC8
:10693000B45E3828A3E6C3E3207CE3B098074A5E40
:106940008C51179CF9F6B77C47C58A4D898EEE515C
:10695000F8C4474B64A5BE6EFA6012BCFC61EE073A
:106960001816A94A1884D397C22BDBE348ADDA3C4A
:10697000A447D9E781F7DFA1DA3C23E49037E24B63
:10698000E4D5808001FBC143298C23AA8BCFE9C1C8
:1069900052125274BAA09825DCF647760B2632C5FF
:1069A00072C5A5872F01F0472AEFA9190E9BD76161
:1069B000C2ACB99EDB54955FF43596F2207D416AF6
:1069C0003472C75F483D18DFC9BCB438D9D9D1DDAE
:1069D00094A083C7C01A452957D0EA008008D71B66
:1069E000C9EADF0698A0B6D60D3A1082C2DD4AC0C9
:1069F000D80D9934F3026D8D63E34A63766F5CB012
:106A0000E59878694A22E348E2CBEF408F8FD77050
:106A100068D3476BB03DF2C3E33F3006A9B9F1EB51
:106A2000EF72215DC599A0A64ADA051F2D98BD48D1
:106A3000BAFFA8D5C635552ED041718977CAF9E37A
:106A40008F5AF8DF73FC1965EA9BEB7737D772979B
:106A5000D244200D5D4CD886AA1A66F0F2BFFCFD28
:106A600076887B5F26CB4F5106C8F7CA243873F06F
:106A7000FBE7FD0AADE9C5F5FD5DDAFCB0E0FDB070
:106A8000DABDDF7D4380D14E3479C9E5673A06C768
:106A90001F850323096903BC96D74AC499C8589433
:106AA000315EB8137C328D87AFCA56629191F0DCAB
:106AB00069B4953858722B1FD1BF11F8CDAB2E1B7E
:106AC0007B27C642E84E6EEA96D1EBCD3B0D1C1FEC
:106AD00033CF0C84395D28811E9BA48E4012D4C410
:106AE000F4B5E2DEA4E2B942FE4CAB58631776601F
:106AF0002379D6CDD68008756D51AAE2C86551C8F4
:106B0000FEE8BFCCE215A25982E4086389E55EF68F
:106B10004EDE5E564EA20AA154D86D4FA8C41A2F5D
:106B2000155E5C759673298A7CCA69433854890757
:106B3000C2AE738D2594305A748D3BE28190E38D03
:106B4000E1417646D11E785CA67E79DBA6659C285D
:106B5000D8440A4C3A400D5E237AF8F81556AFED4A
:106B6000F200FFCCDDEC6161727FD7317B3109F03F
:106B70000AC5F6C8412EBD22681919F48DB1F32F4C
:106B80002EBD05C2AAD79C595FE8A99CBBD49FD152
:106B9000E983E38C27623E72CBAC64B8BE7E60B3FF
:106BA000248771CC1357D40DC315DD7F76560EE1C3
:106BB000E0AA62D0AF989FCDCE888C94EC1402747A
:106BC000B918391B2C5F23D7D0EA123C005F5E2432
:106BD000614BFFB45748699E187EBA104677B0F0F3
:106BE000B38C6D16DADDFF03DDD05E5E91EA78D7F7
:106BF0000752A35FBBD630632E9B91D576C63CE38C
:106C0000EBD8B4DA66402D65D9EC18F0B8B41B3077
:106C10008D127B19C0FB809570EB24B7127839C8B0
:106C2000EB5113F067638821F033F8558E41CB5F49
:106C300097A670AA2AC02D7EB738D97E057923A4DD
:106C40001A999F1A2E9469106E5FF09EC22D39C258
:106C50006F21CAA44B3EDF09D84B84CBF7196E02D3
:106C600085BBCF59FF6EB6226392687C7C5215C4F7
:106C700020D948CF9D65BCD567B7284AEFC0AB4E39
:106C8000DC4887383B38B419DAA2B92F48004B26C4
:106C900012011BB41FF55956A2E5CA25CEB47FF5E3
:106CA00081E003CA062761B4C0B9AF1E9D1B689777
:106CB00038CFBFE131A6D7FB9520278B4B6050EA38
:106CC000A89C8B3D76E9411AB796538C8B29E985B0
:106CD0001279EDCB2E8181C922C4055B6423C81AC9
:106CE000BFF92FA8A161609D6C8C6E80FA68444B3F
:106CF0003DE53978F7E014F0BDD363749A4BD5F5D0
:106D0000119CB4F3C12F23ABAFDB177B7376D9C5CE
:106D1000B1B5F0F48CF88E40DA590F4AF5AC66EC58
:106D200046B267F66D30CF5134B4DC114DD3C15447
:106D3000448CD2B31094CDC369AD88CF24AA5A62D3
:106D4000CCBCDD48C0B34288FCAF3A729B9CBC7798
:106D500012521D5965661E149FC566C024074FF266
:106D6000C615D0DF48B0E4F1CD3891E40879BCC253
:106D7000511C9642CA8F4D970536E1C31398A7144C
:106D8000CE6D7AA026A1D7922DFABF2FA40A442D4A
:106D90004F10186BBB0D39BB6C53C179AF7036887F
:106DA000D9723E5049D312E4D7B348C3EBAB9597A1
:106DB0002C7B94F8F3D00B0F1C4E9ED8E0AD662DC3
:106DC0003C7F12A2BF948B073808747D9D6E881497
:106DD00064219C7E6C27CB181624B8F3776F114E74
:106DE000AFA589D6E7DB6A538560897252FDC50578
:106DF0005B879EC93FB56B74730435AF90600558CF
:106E00005448BCC14669142874CEDC794C41E9D899
:106E1000CB82FE67E774F1BACCD53B4FD5E9E07978
:106E200043F860160B4CB5440A6DE663B2D8F275B0
:106E300058C8FCBEA83586BC7DF4ACFB6D4A5A44EC
:106E400035D4FBAA924E146B088B7695AA27B4D63C
:106E50007E93EB1CDDC4CADC02D1FDF8862619A1A5
:106E600010164678594086B30324AEE97B1C572E92
:106E70007048913A041ECB32C424F1E1890E2B579D
:106E80006CDA999D827E3354DE58DFC0DA1B02EF44
:106E9000D3CDE7B26612F4C84EBD5241773CF90437
:106EA00030C0A157525BEA4C609755EE056519CD8D
:106EB000360674D238F3022DB59759A295D81CC85E
:106EC00005EDCE1DB97831C1D1CA36E62D66A5D102
:106ED0007B13F5F38E5CBCB7979ED3F79EA897986B
:106EE000CF04DDD0F717A09883C7AAD25D42190955
:106EF0008E6AC1E5BC0A41C0D0EE39C374BDF11839
:106F00001B6AFC599320FB757C6D476BB010B28DEA
:106F1000BCBCFAAF2FD40FFEB0455C0F41696E6068
:106F2000626494FC68FD42AA198E31194E3BBF621F
:106F30001A620418700D77452F69DFA1DF9DB4A692
:106F4000D36C3CAB9D38849B26B22802957F82DAB5
:106F50006777C1B706767112DB8E02899D86FDDBED
:106F60009874D59F3318AE7EE95E6722450DA06EFA
:106F7000050AD0859BA1C6BAD0404A6907A0E29B0A
:106F80000CB46E3D795B85C4B045BE1CA5DC83E0C6
:106F900091284FF9550A0644E177AF4F7EF0066815
:106FA000070A524B628C975721EFB06C7E0794977B
:106FB00026E86D4A19500CC84534EB2869308D110C
:106FC00053499119D8E7924A961C515A7F32589EDC
:106FD00059BAE5DBFC8A2C87A929B0304C3747B178
:106FE0002AB4D1E965C87610DA6407AED9564050A4
:106FF00073F63DB97D0597332F1DBE6FF2C197E53E
:10700000B64668845EB510999CBD56B344EDA6E8BB
:107010007561891C76045B8D6E651A9CB2A7FE842F
:1070200035095F1B890FF76C35B13DB0BEBB055EFE
:1070300004928C9866329D7EF4F8EDDF5B981C37E5
:1070400076ACCEADCE4C6482F828C574E207D2BDD2
:107050006067196CA7C153B7F9AF87705663B4372F
:107060004FF7694B4E44494060D01561BEEFEDF4D7
:10707000E01D255197460D1523791DEA5BDF746FDE
:10708000AD22645C7F327FF99E7B4B0AEC6C58D555
:107090007347BD5A93DE7F8808CF47B8E8763E1F16
:1070A000F1DA1CF9CAA2529BE2F19D41F971FA573B
:1070B0001B0A2A8CD2E1FB91B8B0770D01D0386160
:1070C000681FEA23638C3D0C46294AF711E22B44E2
:1070D0006EC4CF0E179C55FC47EA9AF09B90E2498C
:1070E0009A20210106AD4FEA06FC52C27B7AEEF5EA
:1070F0006DC03A85822BDD8B3F00FF92A1DD4745B5
:10710000EDC3AEE7D18933B50C967FF15F1A024C1F
:107110007AEDFAC6664AFEF08918808AB01A513CA8
:107120001D14BE57BDE2BA161A0184C448EC98CFAC
:107130006E039503B5BB5F1D1E7D64F40A143E8289
:107140006EA6E02A0B7ACAA5C4F878E36F0F694EE1
:10715000597EC2824000BC2F7F7773B3DDBAFCA991
:10716000A9D5477C34BB28494358A96F77FA7E38A4
:10717000FE561B7B9B0EE3EF56C68B912D4FCC45E5
:1071800046750C1314D34FFFBAF3735A2D3071E0C8
:10719000EFD846018FF5C257A8BA8B53231E506F04
:1071A00044FFCE76741D3473BBEAD36287F75BBBB2
:1071B000934426BDF45B516DA046F25F0B05EFC60C
:1071C000CC344EEACAC298EEBCF3F76F2B9D782DF3
:1071D00046F98949BD7C45E67BEFEAD555A9228E63
:1071E000D31863603A90AF3DE84A7EF83C5FCA54DA
:1071F0003C38C77414EC67FA56174AD1FE51E5D3F0
:107200001EEB4CEF48B03B51D981850C32C584F15F
:10721000EA191301944282CCB1B35662BB0D2B1A0A
:107220001B9C73615C978F3F3C1ACC27A624EA9085
:10723000064A26FE14734436AA4758869E27024AF9
:107240005317DB91629E681BBD238550D54EBC222F
:107250004D51D1E41470292AB232E229DBF3C67011
:107260008EE177C65F3CCD09732B02B82F65BB2139
:107270008C73AB3F03D9E5DDB788BF15231E0F48DC
:107280004C142DCBE06F0A94D381C0EC07BBB954EA
:1072900060348FCA35486984383070E8FEB5F14BE8
:1072A000309DFCD07BA3B16BD709509D87F1E1D213
:1072B000808A59EB3B5EB9BC685CF5592B918165BE
:1072C00075E7E75ECC52824B9EA717146D4ACB98A8
:1072D000A8113492E89976F1BA9C098F1B7C40F989
:1072E00050061A045F8B62898942C45B147D75EE77
:1072F0007BD1904577E761053534E4B02878753265
:1073000098A21EA6B4C776C03BB6A35E9087250E92
:107310006A3B72CABC24C075236136FDAB152FA72A
:10732000F518631E958BB78F434D5E339919A4539F
:10733000B8A2FAE3885FD761D705A5788AA0196F4C
:1073400020DAE324CA75A7520C78006269D651840A
:10735000D73770B738B6CC6398CF24118949D7E9AD
:10736000B7DE2F494C85042BD350593391B795A3E1
:10737000809F0F0D003B0F1561894F9C7AC2685D9D
:10738000A6585813D2ADADED354857410C466B1297
:107390000B731344067F773066C10679D1A668E285
:1073A00039756B52DBE3F94E881486D39783210F2E
:1073B000824F596B6FD320797100295DB838587BA3
:1073C000B33DA6CFC6E35B9C1FF9D400C6889C06DC
:1073D0002795FE156706288D2585FE1D48893AFFED
:1073E00009F43693CD5E58F43BBEFA0494B5A44C30
:1073F000062C1884667E51CAC4A2C2F276E1600CE3
:1074000014E1A92DC631982635BFE02C5476A4DAB4
:10741000C79969F7E031B0A8D4B61759CC90995EF6
:10742000E843A586A8A79C79DBE233EDCF85F84336
:10743000A9CAEA723F60F008E9A7C847B3DCFB8A33
:10744000E6DB1972F0016B43D987B36928F6942CF7
:107450000D2F2B752286FB860953469D510315324D
:107460000B1A1DE6200243E2FC0A0E06385050209B
:1074700080ABB712D46C70B53D4BD772B3713CCDB5
:10748000CD68666E3D974A2865253F87B64ACBB6DC
:1074900078214318281DC65627538E8CD19A76D54D
:1074A000C77E50C7A9C7BD0B5262102D6177B7E0E8
:1074B0003D078CF2174885700D14A3FBA2B5B224CA
:1074C0002725D000F3D2FE29BFF22224A2A4B8AE11
:1074D00064EE0330C9980C31BB93ED5B52C80EDAF1
:1074E000490EC70A2CC0B7AB3F894159AF0E1A3DB0
:1074F0007B6864EAD5E91735822B023A2B59203A8A
:107500003BA89953CE6BE5766BC573C5E7F668AAC1
:10751000C6C12AF2B5A833A31F45A6A28B112E55CA
:10752000AC300DF70FA7181E5C105AA9BA62D2AF83
:107530009BAE7A2A3D64F9E99BF87D6CE37E247763
:107540002E9E3CF7467C4131EEAAA2109263A36BBB
:10755000219FBC7A0D8A2F6708240A344B5255FBB1
:10756000377C8849D3FD9603FF4C14D8EEA37ED513
:10757000E810AB20149147997A2B7E8085FF7075B7
:107580008B5919CBC2BC13D77938FE4A58D8956E9F
:10759000FE478F2A707A07A3C79EFDA4FE2EAFEA8E
:1075A000A257AD1ACE6BB48543CF08FDCC7261D91A
:1075B000A1F5CF2152AF7A2C914897C68754C2AF1C
:1075C000B0289509AE277A0C04550F826A82179B62
:1075D000AF7F8A346A3DF9130AE10F04FAC333C15D
:1075E000D422A9AFFA112B72CECADFA6D66B66538E
:1075F000DE5AF2E3E4DE8DFAB19247BF7AA4702539
:10760000ECFB924BA294C599D57B73096994A06D4C
:10761000846E9999691FCA32443227A8DE3A633AC8
:10762000092A9120F130E03244229FFC22C8FF8DCC
:10763000E213E1AB67CF041A9B473F2AAE4CFF87AA
:10764000A8703454A9BE58BAF81AB302D839B00E8B
:1076500084B5DB1B30B6AD23207DD5DC4B35C85D52
:10766000DC915E31617C69327D529D39DABCD2E9B0
:10767000FEB97709035BF9FEA4CA46853C03D8D25C
:10768000C4D4A65CC9E7B4E5012A605D72B482F592
:1076900073719035CA7EF59430DC1F8B9F2527A42B
:1076A000243AE08BDADED6C105E2E6E99A27A28821
:1076B000C285D230C8E2BC580004A99D8F0A5C99EB
:1076C00041BD0D19CCF487D2ECBD274AACD9BBBA69
:1076D0001242FB423F73ED5B16457BF4D81312DF79
:1076E000C9E5787B25990042EDB57885EE3BB195EB
:1076F000C2E70F60633FB5F4636AADA2795DD882DB
:10770000D9BA823F0CA6AFF9EE7F35AB58A5CA9E19
:1077100078FCC7613158E42B431181F68E764BD348
:10772000C079E08C49E6E37F27D61BF576FA89AC71
:107730004E9824BAD63220F1434F4E5F6213BC3BC1
:10774000ADD5A1F3587369BF653D00CC2D38A0C4F9
:10775000014F1DD8B6852B3C5D08D84B5F595AF3B5
:10776000605012D9029DAF5F28B0B3D89C77001645
:1077700017E33697D35F5D87BAC1B772AFF9FA7F67
:10778000F1876E5C208AF1E9FCA602763CD71A7379
:10779000FEFA75539219BF699DB3E92992318D1193
:1077A000B240C80115C186CED3783D64E527DDDF40
:1077B0001FA6E26AA3F267D488EBA390EB24E3CB85
:1077C0004ECB55994F7A9E6157FD2A6BBAE02B0E2E
:1077D000C0B2B7951A0FAD18315AF5E3396B675A35
:1077E000E58A690BFC97A1FD1D8656C671FE2785AB
:1077F000155531DA04A9ABC36D0661A6035C8DB6DD
:107800007EE9EC999A73643CDA7EA0FEECB3351FF6
:10781000221C731BF8E55ECD55A8E4522F7383B686
:107820006BB47F008E44FA752659BD49DEF78D6E24
:107830005E8081FF63A61830144CBCA5C95BE4B21E
:1078400077649C85CDC654C08FF4BCA03F93578607
:107850002FF02248FF201CE5004FE6DBB7BECFB873
:107860008C99914DC75A2FB8547731241C80A08829
:10787000D7C1CAB4605042340117FF546423515435
:10788000F797EFD0E21E4A0943E65389B9C212D1F5
:1078900024FED872A1BFB152575E92FDE0548A52C5
:1078A0003D15BFEB98B03A153C6F160A51CFE57AFB
:1078B0009F2DA75C6B6FA96FDB1C61BCE8897DD233
:1078C000F9FB274B1EABA18B3C3BEDD5B183F5BD3E
:1078D00097E2C54AA11210C6A990AA89E9B655E156
:1078E000452CADA74A9A933E6F4CA6B1289CC4CDB7
:1078F000A6D5CA7E2C9E29F9E1CEE3C56B0404957A
:1079000032CD66203CBFAF826D46A627F50B3C46C4
:10791000FE43DA3FD059FABE16A7E996482ABB893A
:10792000468689DFAFB2892BB4236A78E0474AC91B
:1079300008558AFA00BCDF5450A997710D58D840F9
:10794000FE85044FE77D51B4C478ECFFDC1392A3AD
:107950004EEE9EBEACA449E4D0EA722324E57BD16E
:107960005F1817A4CD55A36F913D7D8633B0E15AC2
:107970005212A722DE11A84A305BF9542811EA619D
:10798000132294DFA15F11D1041733E45F13A650D3
:1079900001111B6FD59A93CB3A06AFECAF69CFD7E5
:1079A0006A78ECC0B9BAF2A2A51750EBA8E7EE4E80
:1079B000CEFF9FCB8D470932177DA62D39AA473DB3
:1079C000267AD8133C31518E91169C50DD6365ACFC
:1079D000C0A64D6B3EEDB01EDB52BB8E8E03791000
:1079E0005118EBCE4DB59681469BE7725833711412
:1079F0006D8A5E508FB7AEDF92663DF4E0D948CB1A
:107A0000E68E4E3E4E714C64B726DA09D3881FCA03
:107A1000057D1536AEC34936DBD624F3CA9A11E28A
:107A200043A491AE6FD3FC9C7F6D52753F72CED351
:107A3000D23DD278A4761E1B1DEA29AE5AA980A099
:107A40007825D9D6D9A52ECE8BFFF0AE25983DC38B
:107A50002BF55C0F4F39BB80385341EA0C415D1E5A
:107A60009FE484D8F473F4992C2C44DED4BEB6F091
:107A70001370679D7078FF04CEF0AFC9F97FBB3CEF
:107A8000486C2A06BC4C9CEADAFBDEB89BBF13CAE2
:107A900051F2A5A188E33B9C365FF5E180E2349486
:107AA000C42FCBC9BA1943BAB7552659DE14FC3EC8
:107AB000F987E0058C446413A595F58EECAF9DAC79
:107AC000EAEE88CB982C6FC074272DD4850A7B17DB
:107AD0001B20549BA3E79BA703BA6D0B4B67C69073
:107AE00062E8A610E76960A22EEAB42F0CF28E704D
:107AF00008E14922194BF4F8456B359502567D7221
:107B0000F7EE031A27E4161237943838E1C764BC3D
:107B1000C05FF66075F3CFB1C5CCAF18D51F9D1609
:107B20006DB30BEA6D2E68A85F0A5C82920BF515A7
:107B30008CEED1A08DCEB5E31BD5EEF8039776B8C9
:107B4000ACB7A0EA22FE25B9DC1125CB226C36B9F0
:107B5000ED01F1F25FCAA28604F324609359FB5150
:107B60005DE4EE57C76FC2F12579941CA909946AA8
:107B7000DD42D0FB5658783539F62321B08A26D31A
:107B8000FA8B15A32F6419148EC59797991C7B70D7
:107B9000257D8BA6266789743EFC782896765F66DD
:107BA0003ACA0550F8D4DA7897D2BF92F858A5139C
:107BB0006DF98025B2B15FB84E28A3D19494110C11
:107BC00040CA24BAD633AF4C3E6913A4AB761BF53A
:107BD000C0640B829D4FAA03ED47CCEC16E2B9BFFF
:107BE000F7D353F25717E050842856C180C1EB6990
:107BF0008BCEC3B01E2F1EB58784E9497F2938D2AA
:107C0000B316A96EC7C4EDD10E83716803542E322A
:107C1000A7D8580A10E2940BE4C924865B7A270A95
:107C20000A801518689EB5AE10986F3B3A80987D13
:107C3000B3FA20E3B15CC08A0C5DE9F957FED25D6E
:107C40003FB077D08A2066A9172908189CC1C0596F
:107C50006049E7BE939291678555A11B04CA1A72C9
:107C6000A25D16F60304050A08060BFF0209070DBC
:107C7000010C00FF2025692025692025692D256933
:107C800000202025633A256900202020205F5F7CAA
:107C9000002C00610044697370206F66660D0A0055
:107CA000555345520046004700424547494E005251
:107CB000414400442E4D590043005052474D005559
:107CC00053455220202000662020006720200042DB
:107CD0004547494E202020202000524144202020AA
:107CE00000442E4D592020200043202020000D0C60
:107CF000205A363C00000500000003072061703B5D
:107D00000000FFFFFFFF4D000000B43F0000000037
:107D1000000085100000CC3F0000D13F0000CF3FA5
:107D20000000FF00000069080000DB3F0000E53FA5
:107D30000000833F00000000000089060000F73FBC
:107D40000000D13F000003400000000000002907B0
:107D5000000005400000D13F00001140000000007D
:107D60000000C108000013400000D13F0000344073
:107D70000000000000005106000036400000D13F26
:107D80000000FFFFFFFF0F000000F40100000401EE
:107D900003010201010411040F0417041601180164
:107DA0000000BF7C0000C77C0000CB7C0000CF7CC3
:107DB0000000A77C0000DA7C0000E17C0000E97C88
:107DC0000000BA7C0000081C242C4448586C740540
:107DD00002050804080B0804040501050409080944
:107DE000040608070206020402060106040701034E
:107DF0000803040C080D020C0203020C010C040D14
:107E0000010D080D0408020808070802020704080B
:107E1000010804090209010A080B020A0201080A02
:107E2000010A040B010208020410081102100211D9
:107E3000081001100411011202120113021308129A
:107E4000080F08120413011304140214011502157B
:107E5000081408170814041501150417021701194E
:107E6000081A0219021602190119041A0116081635
:107E7000041B021B081A0818021A041B011B041811
:107E80000818040B0420202020202020202020007F
:107E9000000001000000A07C0000A57C0000A77C81
:107EA0000000A97C0000A77C0000AF7C0000B37C30
:0A7EB0000000B87C0000BA7C00005E
:00000001FF
